S31500000400FFFFFFFFFFFFFFFFFFFFFFFFFEFDFFFFF9
S315000080004816002069850000718500007385000010
S315000080107585000077850000798500000000000066
S315000080200000000000000000000000007D84000049
S315000080307D850000000000000585000055850000D4
S31500008040838500008385000083850000838500000A
S3150000805083850000838500008385000083850000FA
S3150000806083850000838500008385000083850000EA
S3150000807083850000838500008385000083850000DA
S3150000808083850000838500005992000083850000E7
S3150000809083850000838500008385000083850000BA
S315000080A083850000838500008385000083850000AA
S315000080B0838500008385000083850000838500009A
S315000080C08385000083850000838500007B8C00008B
S315000080D0838500008385000083850000838500007A
S315000080E0838500005DA6000083850000838500006F
S315000080F0838500008385000083850000838500005A
S315000081008385000083850000838500008385000049
S315000081108385000083850000838500008385000039
S315000081208385000083850000838500008385000029
S31500008400DFF80CD007F008FA004800470FAA000072
S315000084104816002080F309887047EFF309807047FB
S31500008420684680F3098804480078C00714BF022014
S31500008430032080F3148870478C090100DFF818C008
S31500008440EFF305831B0618BF6047EFF31483DB07C2
S3150000845008BF604700DF704787000100DFF818C0DB
S31500008460EFF305831B0618BF6047EFF31483DB07A2
S3150000847008BF604700DF704791020100EFF30980F3
S31500008480816911F8021C39BB90E80F10E047EFF341
S31500008490098C194B93E80600914218D059B10CB4D7
S315000084A04FF0010381F821302CE9F00FC1F824C008
S315000084B000F077F90CBC1A60D2F824C0BCE8F00FC3
S315000084C092F821308CF309881BB192F82000CCF881
S315000084D000006FF0020E704710B5084A126891420C
S315000084E009D8074C54F8214090E80F10A047EFF345
S315000084F0098C8CE80F0010BD14E1FF1F98F80000EE
S3150000850098F8000007F0B4FF114B93E8060091427B
S315000085101BD00CB44FF0000381F82130EFF3098C27
S315000085202CE9F00FC1F824C000F03BF90CBC1A602E
S31500008530D2F824C0BCE8F00F8CF3098892F82130F9
S315000085401BB192F82030CCF800306FF0020E704765
S3150000855014E1FF1F08F07CF9D6E7000007F092FD52
S3150000856008F076F9D0E7000006488047064800473D
S31500008570FEE7FEE7FEE7FEE7FEE7FEE7FEE7FEE7CD
S31500008580FEE7FEE78D850000018400004CF22050D6
S315000085907849C8814DF62810C8814FF4E9700880E3
S315000085A04FF488107449486400207449087074496F
S315000085B00873242048709A2008700846C07800F096
S315000085C01F00C870032008710020487100BF6C4866
S315000085D0807910F0020FFAD000BF6948807900F068
S315000085E00C000828F9D1032065490871402048711C
S315000085F000BF6348807910F0200FFAD000BF6048B2
S31500008600807910F0400FFAD01A205D49087000BF3B
S315000086105B48807900F00C000C28F9D100BF58485F
S31500008620807910F0400FFAD04FF4004055490860A9
S315000086307047534A127812F0C00F66D1504A5279E9
S3150000864012F0400F51D14E4A127812F0040F18D191
S315000086504B4A127B12F0010F01D14B4801E04FF457
S315000086600040474A1278C2F3C20301229A40D1B2AF
S31500008670B0FBF1F0424A527812F0300F03D04009B5
S3150000868001E04FF400403E4AD27802F0E00212F0D8
S315000086901F0F28D15211082A25D2DFE802F004085C
S315000086A00C1014181C2000EB8002D0011CE000EB1B
S315000086B08002100218E0C0EB0012D00114E000EBBB
S315000086C08002500210E04FF4377250430CE04FF432
S315000086D0B762504308E040F69502504304E040F686
S315000086E07132504300E000BF38E0254A127902F0AB
S315000086F01F02511C244AB2FBF1F0214A527902F0C2
S315000087001F0202F11801484328E01D4A127802F0C0
S31500008710C002402A11D11A4A527812F0010F02D132
S315000087204FF400401AE0164A127AC2F342030122BD
S315000087309A40164BB3FBF2F010E0114A127802F0A1
S31500008740C002802A09D10E4A127B12F0010F01D114
S315000087500D4803E04FF4004000E07047064A526CB3
S31500008760012303EB1272B0FBF2F2094B1A6000BF51
S31500008770F3E700000020054000800440005006405A
S315000087800040064008ED00E000127A0000093D00B6
S315000087900000002000BFFEE7704700BFFEE77047FD
S315000087A070477047232000F01F02012191404209C3
S315000087B04FF0E02303EB8202C2F8001100BF7047BE
S315000087C00820FC490870FC48406840F4A020FA499B
S315000087D048600846806C20F00F008864002088649A
S315000087E00846406B40F48020486301DFF348007878
S315000087F040F08000F24981F80C0100BFEF48007894
S3150000880010F0800FFAD1EF48000AEF490870ED48E2
S315000088104FEA1040EA4981F8B000EA484FEA106092
S31500008820EA4908704FF0FF00E54981F88000E84802
S31500008830006808B1042000E0002040F01900E44977
S31500008840096809B1022100E000210843E1490870E6
S315000088504FF04000DA4981F80001084690F80C0113
S3150000886040F0400081F80C01704758B1DA490978A8
S3150000887041F00101D24A82F894104FF01001D74A14
S3150000888011700DE0D449097821F00101CC4A82F833
S315000088909410114691F8081121F0100182F8081180
S315000088A07047012005E00022C8490C3101F820205C
S315000088B0401C1028F7D30821C24A5180C84951608C
S315000088C0C821117000211172C54980315161002201
S315000088D0BC49CA610D21C34A11704FF05531C24AD5
S315000088E01160B74991F8941041F00201BA4A11702B
S315000088F04FF0FF01BD4A1170BD4A117002F104022A
S3150000890011704FF00001BB4A11707047B1480078F2
S3150000891040F02000AA4981F884007047AD480078ED
S3150000892020F02000A64981F8840070474CF25030B0
S31500008930B149097811F0020F13D0A749097841F01F
S3150000894004019F4A82F8941000E000BF0100A0F1E4
S315000089500100FAD1A049097821F00401984A82F869
S3150000896094107047704719B900F07F02A14B1A7036
S315000089707047704710F0800F20D000F00F000121E3
S3150000898001EB40029140984A12681143964A1160E1
S31500008990022101EB8001924A02EB8112022101EBD6
S315000089A08001884B03EBC1014A600022022101EBE2
S315000089B08001491C03EBC1014A6034E042000121F9
S315000089C09140894A12688A4387490A6079490A5C54
S315000089D000F00F01002303EB81017A4B03EBC10189
S315000089E04A8000F00F01002202EB81017C4A02EB73
S315000089F0811200F00F01002303EB8101714B03EBA1
S31500008A00C1014A60882200F00F01002303EB8101B7
S31500008A106C4B03F83120002200F00F0102EB8101BC
S31500008A20491C03F83120704770B50446A578A6881E
S31500008A30A07810F0800F01D15E494E552846FFF709
S31500008A4099FF70BD704710F0800F0AD000F00F003C
S31500008A50644911F8201041F00502624901F820200E
S31500008A6007E0604911F8201041F009025D4901F85C
S31500008A702020704710F0800F0AD000F00F005949EF
S31500008A8011F8201021F00502564901F8202007E0D0
S31500008A90544911F8201021F00902524901F820200A
S31500008AA0704700F00F004F4911F8201041F0020204
S31500008AB04C4901F82020704710B50446494804F097
S31500008AC00F0110F8210020F00201464804F00F02C1
S31500008AD000F822102046FFF74DFF10BD7047F0B595
S31500008AE003460C46002503F00F06002707EB860118
S31500008AF0344E06EBC10670883BB9324E16F831602B
S31500008B00C6F383060D2E00D10125002205E0344E62
S31500008B1006EB8116B65CA654521C8242F7D3254E4C
S31500008B20F65C284F07EBC1077E804F082E4E36684D
S31500008B30FE4006F00106234F17F83170C7F3801781
S31500008B40BE4211D145B1A67936B9274E366826F010
S31500008B500106254F3E6007E04F080126BE40224F22
S31500008B603F687E40204F3E604F081F4E3668FE40ED
S31500008B7016F0010F0BD04826124F07F831603E461B
S31500008B8016F8316046F0800607F831600AE00826DC
S31500008B900C4F07F831603E4616F8316046F0800605
S31500008BA007F831600C4E367826F02006044F87F819
S31500008BB09460F0BD08000020008004400C210740AE
S31500008BC000200740000200209C200740B4200740F8
S31500008BD00CE1FF1F8420074094200740082107402E
S31500008BE0A0020020C020074004000020802007408B
S31500008BF08820074098200740E8E0FF1F70B503462D
S31500008C000D4603F00F03022000EB8301844E06EBB2
S31500008C10C1067280002405E0285D824E06EB8116AF
S31500008C203055641C9442F7D34E087F480068F040E4
S31500008C3010F0010F04D08820794E06F8310003E0C9
S31500008C40C820774E06F831004E080120B040764E17
S31500008C5036687040744E3060104670BD73480078B8
S31500008C60734991F8A41040F2FF7202EA012140EA2A
S31500008C70010070476F48006870472DE9F0416E4863
S31500008C8000786B4991F8841000EA010515F0010F90
S31500008C900ED0FFF706FE04F0B8FD6848006820B164
S31500008CA066480168042007F0C5F90120624908708A
S31500008CB015F0100F0CD0FFF729FE6048006820B1B0
S31500008CC05E480168102007F0B5F930205A4908704F
S31500008CD015F0200F0CD0FFF721FE5848006820B190
S31500008CE056480168202007F0A5F92020524908704F
S31500008CF015F0040F0AD05148006820B14F480168AA
S31500008D00402007F097F904204B490870022D13D133
S31500008D104B480078474908604848006820B14748F2
S31500008D200168802007F086F9FF20454908704FF05A
S31500008D3002003F4981F8800015F0080F6DD04148C8
S31500008D4000784FEA10143A4890F89000C0F3C00635
S31500008D503C480078C0F3800754BB710004F00F0054
S31500008D6001EB8000012101FB07002D4911F83000BD
S31500008D70C0F383000D281BD12B48006820F00200A9
S31500008D80294908602648007E20F08000244908769C
S31500008D900846007C20F0800008742B4850F8240018
S31500008DA0C0B3294850F82410022007F043F931E0F7
S31500008DB0710004F00F0001EB8000012101FB0700A8
S31500008DC0174911F83000C0F38300012809D11E4865
S31500008DD050F8240028B11C4850F82410042007F04D
S31500008DE029F9710004F00F0001EB8000012101FB5D
S31500008DF007000B4911F83000C0F38300092809D198
S31500008E00114850F8240028B10F4850F824100820C3
S31500008E1007F010F9082008490870BDE8F081000045
S31500008E2000020020A002002004000020A02007402D
S31500008E300020074010000020802007400CE1FF1FA3
S31500008E408820074090200740ACF4FF1FF648806B4F
S31500008E5040F40060F44988630846406B40F40060C3
S31500008E6048634FF44070F149C8600861DD20F0495D
S31500008E7008740846C07840F00C00C8707047704708
S31500008E80EB48C07820F00C00E949C8700846C07865
S31500008E9020F06000C870122001218140E54A430994
S31500008EA042F8231000BF70472DE9F04304461F46E1
S31500008EB000250026DE48C07820F00C00DFF870C3DD
S31500008EC08CF803006046C07820F020008CF8030080
S31500008ED00020DFF864C3CCF80000CCF80400DFF80B
S31500008EE05CC3CCF80000CCF80400DFF854C3CCF81F
S31500008EF00000CCF80400082902D0092900D0082176
S31500008F000839012A03D101250126491C04E0022A59
S31500008F1002D101250026491C022902D10021002583
S31500008F200026080140EA45003043DFF804C38CF808
S31500008F3002002001DFF80CC3BCFBF0F3BC4800784C
S31500008F4020F01F00C3F3042C40EA0C00DFF8E0C257
S31500008F508CF800006046407863F307008CF8010047
S31500008F606046C07840F00C008CF803006046C0787C
S31500008F7040F020008CF8030012204FF0010C0CFA90
S31500008F8000FC4FEA50184FF0E02909EB8808C8F8B2
S31500008F9000C100BFBDE8F08310B50246086840284E
S31500008FA001DD402000E00868034616E000BFA34844
S31500008FB04068A24C2468A042F9D0A0484068401CF2
S31500008FC09E4C606020460079401E00F03F049B489E
S31500008FD00830005D40B202F8010B1800A3F101034E
S31500008FE0E4D10868402801DD402010BD0868FCE790
S31500008FF010B502460868402801DD402000E00868F8
S31500009000034616E000BF8E4840688D4C2468A04297
S31500009010F9D08B484068401C894C60602046007936
S31500009020401E00F03F0486480830005D40B202F85A
S31500009030010B1800A3F10103E4D10868402801DD03
S31500009040402010BD0868FCE770B5054655B1DFF84D
S31500009050F8C100DF7D4908607D480068416800204E
S31500009060884710E0DFF8E0C100DF04467748006873
S31500009070201AB0F5967F03D3012001F048FB02E0E9
S31500009080002001F044FB70BD00206B490860486079
S315000090906A49086048606A49086048607047F0B5E8
S315000090A002460B461968084600BF634C6468624D69
S315000090B02D68AC42F9D10DE012F8015B5E4C2678C2
S315000090C02468641C5C4F06F03F063C6007F1080408
S315000090D0A555491E0029EFD15E4C246844B10024F1
S315000090E05C4D2C60524CE47844F04004504DEC70DA
S315000090F0F0BD10B50146514A1278504B1B79D21A71
S3150000910002F03F024D4B1B7903F03F044B4B1B789B
S315000091105B1C03F03F039C4201D1012300E00023C6
S3150000912042EA0300402801DD402200E002461046E4
S31500009130086010BD10B50146414A1278404B1B79B4
S31500009140D21A02F03F023E4B1B7903F03F043C4B20
S315000091501B785B1C03F03F039C4201D1012300E016
S31500009160002342EA0300402801DD402200E00246D7
S315000091701046086010BD7047F8B504460D462078C5
S31500009180802810D101F0F3F80746381D06F0A8FA3A
S31500009190C6B2802028706E703246391DA81C06F0B3
S315000091A07BFAB01CF8BD2078812814D16846FFF7F9
S315000091B0C1FF00983E2801DD3E2000E000980090A7
S315000091C081202870009868706946A81CFFF710FF78
S315000091D00098801CE6E7207882280AD1607840B2A1
S315000091E000906946A01CFFF75AFF822028700120D4
S315000091F0D8E72078832813D16078A17840EA012047
S31500009200E17840EA0140217940EA01660123002223
S3150000921008213046FFF748FE832028700120C1E769
S31500009220FF2028700120BDE70080044000B0044004
S3150000923000B0064080E100E090F3FF1FD8F3FF1F67
S3150000924020F4FF1F006CDC028D08010018000020CE
S315000092504C0000201400002010B52749097911F0B0
S31500009260400F23D025490978244A1279891A11F02A
S315000092703F0F12D021494968491C204A51601146C6
S315000092800979491E01F03F021C490831895C1A4AD6
S31500009290D17100211A4A116008E00121184A1160B3
S315000092A01549C97821F04001134AD170124909794C
S315000092B011F0200F1ED018E00F49C97948B21149A4
S315000092C00B780968491C0F4C03F03F03216004F139
S315000092D00801C8540C490B780968491C0A4C03F06C
S315000092E03F03216004F10801C8540349897C11F049
S315000092F0400FE1D010BD000000B0064090F3FF1F04
S3150000930014000020D8F3FF1F20F4FF1F0020704731
S3150000931000207047002070470020704700207047EB
S3150000932000207047002070470020704700207047DB
S31500009330002070474FF6FF74002220462146DFF8D2
S31500009340D4C000DFDFF8D0C000DF4006F4D505F05A
S315000093502AF804F09FF9EFE74FF6FF740022204643
S315000093602146DFF8B0C000DFDFF8ACC000DFC00781
S31500009370F4D004F0F1FFF1E7002902D0DFF89CC039
S3150000938000DF7047DFF890C000DF70470022DFF88B
S3150000939084C000DF704710B500F050F800F0C1FE41
S315000093A0BDE8104004F04DB82DE9F0411C4C1D4FAE
S315000093B000252560B86938B100231A4603211A48EA
S315000093C0DFF868C000DF2060DFF858E0184E0024A0
S315000093D00EF1200E46F824505EF8240038B1002322
S315000093E01A460221DFF844C000DF46F82400641C58
S315000093F00F2CEFD90F4C2560F869002807D0002301
S315000094001A4602210C48DFF824C000DF2060BDE8C0
S31500009410F08100005102010099010100F1010100F3
S315000094200CE1FF1F240A010035930000D908010052
S31500009430ACF4FF1F10E1FF1F5993000000207E4986
S3150000944008707E4908607E49086001207D490870E1
S3150000945000207D4908707D4908607D490860704795
S315000094602DE9F04104460F4615461E46012C02D052
S31500009470032C38D136E026B1012E04D0022E2FD18E
S3150000948000E000BF2CE07248006870490968884215
S3150000949002D16D480078F8B16E486D4A126800EB4B
S315000094A082114022284606F0F7F869480068401CF9
S315000094B06749086008460068052801D10020086051
S315000094C06348006861490968884202D100205E4904
S315000094D008704020BDE8F08101205A49087000BF9D
S315000094E000BF00E000BF00BF0020F3E72DE9F04118
S315000094F00646884614461D46069F022E02D0032EB7
S3150000950038D136E005B935E02078072803D10120A7
S31500009510514908702EE04848007830B14748006845
S3150000952047490968884200D124E04C49434A1268F9
S3150000953001EB82102A46214606F0AEF83F48006845
S31500009540401C3E49086008460068052801D10020F5
S3150000955008603A4800683A490968884202D1012001
S31500009560354908703E4801680120DFF8F8C000DF81
S3150000957000E000BF00BFBDE8F08110B53EE0354A0F
S31500009580324B1B6802EB8311344A2D4B1B6802EBEE
S31500009590831002F012FE2A480068401C0521B0FB29
S315000095A0F1F201FB120026490860084600682349CB
S315000095B00968884202D100201F49087021480078B6
S315000095C060B100201F4908702248204A126800EB4B
S315000095D082114022002004F0FFFF0FE01B480068C4
S315000095E0441C052C00D10024184804600068184962
S315000095F00968884202D101201349087010480068A2
S315000096000E4909688842BAD10B4800780028B6D1BD
S3150000961010BDDFF854C000DF114908600BE00022DE
S315000096204FF6FF710120DFF844C000DFFFF7A5FF0A
S31500009630002001F079F8F2E71C000020200000204D
S315000096402400002028000020290000202C000020F3
S3150000965030000020E20A002058000020A209002065
S3150000966034000020F10101006D09010051020100E2
S315000096700021FE4A1160FE4A1160FE4A116090B157
S31500009680FD4A1160FD49097809B1072100E008216A
S31500009690FB4A11600021FB4A1170FB4A1170FB4A1C
S315000096A01170FB4A11600021FA4A1160FA4A1160F2
S315000096B0FA4A1170FA4A1170FA4A1170FA4A117090
S315000096C0FA4A1160FA4A1170FA49FB4A11600121FF
S315000096D0FA4A1170704710B50446E8480470012034
S315000096E0FFF7C6FFF64801684FF4804006F0A2FC7B
S315000096F001F02BF805F082FF10BD0024002600279C
S31500009700A046DFF8C0C300DFED4908604EE0002246
S3150000971064214FF4E040DFF8B0C300DF0546022DB8
S3150000972030D1DFF8A8C300DF044614F4805F1AD0F6
S315000097300120DF4908703220DFF894C300DFDC48DF
S31500009740007801280FD1CB48007810F0010F04D023
S31500009750D849D148006801F045FA0120FFF7BBFF60
S315000097600020D349087014F4005F05D0DFF864C305
S3150000977000DF06464FF0010814F4804F16D04FF074
S31500009780000813E0B8F1000F10D0DFF848C300DF7F
S315000097900746B81B40F6B831884207D94FF0000893
S315000097A00620CD4908700020FFF795FFAFE710B5FA
S315000097B00020C9490870FFF78EFF10BD10B5C748D5
S315000097C0007810B10120B7490870AB48006801283D
S315000097D04FD0C248007800284BD1B2480078012803
S315000097E007D10320BC4908700020FFF774FF012051
S315000097F010BD05F01CFF00BF2020B94908604FF0DE
S315000098004000B849C1F884004FF0010088644FF069
S31500009810100088604FF0020048640846406940F036
S31500009820100048610846806840F0100088600846CD
S31500009830806C40F0010088644FF0020048640846DE
S31500009840406D40F00200486540F21310A64948609A
S3150000985000BFA648006841684FF00100884701F044
S3150000986065F918B9FFF7A3FF0120C1E70120824976
S3150000987008600020BCE72DE9FE4F05460F46082488
S315000098804FF010084FF0000A00264FF0000B0020A2
S31500009890029001900090032F11D17848007801289A
S315000098A002D14FF4947001E04FF4A470044673485B
S315000098B00078012801D1072000E006208046002616
S315000098C00FE0E01C285C10F0100F09D0012082493F
S315000098D008700020FFF7FFFE4FF0FF30BDE8FE8F57
S315000098E0761C4645EDD3032F11D164480078012834
S315000098F002D14FF4947001E04FF4A47004465F481F
S315000099000078012801D1072000E0062080460026C5
S3150000991017E2285D422807D1601C285C492803D13C
S31500009920A01C285C4E282BD0285D622807D1601C1D
S31500009930285C692803D1A01C285C6E2820D0285DED
S31500009940502807D1601C285C412803D1A01C285C44
S31500009950522815D0285D442807D1601C285C4F2862
S3150000996003D1A01C285C57280AD0285D43287BD148
S31500009970601C285C5228FAD1A01C285C4428F6D129
S31500009980285D42280AD1601C285C492806D1A01C03
S31500009990285C4E2802D14FF0000936E0285D622887
S315000099A00AD1601C285C692806D1A01C285C6E2898
S315000099B002D14FF0000928E0285D50280AD1601C2A
S315000099C0285C412806D1A01C285C522802D14FF001
S315000099D001091AE0285D44280AD1601C285C4F283A
S315000099E006D1A01C285C572802D14FF002090CE0D2
S315000099F0285D432809D1601C285C522805D1A01C8B
S31500009A00285C442801D14FF00309E01C285CC0F310
S31500009A10400001902819C07D0006144908602819E5
S31500009A20807D096841EA0040104908602819407D98
S31500009A30096841EA00200D4908602819007D096877
S31500009A4008430A4908602819C07C000211490860C9
S31500009A502819807C096808430E4908600846006892
S31500009A60C01C0860014843E00DE1000078E0FF1FDC
S31500009A707CE0FF1F80E0FF1F88E0FF1F59E0FF1F0B
S31500009A8054E0FF1F99E0FF1F9AE0FF1F9BE0FF1FB6
S31500009A909CE0FF1FA0E0FF1F8CE0FF1F84E0FF1F7C
S31500009AA085E0FF1F90E0FF1F91E0FF1F94E0FF1F7E
S31500009AB098E0FF1F280C0020A000002058E0FF1FA0
S31500009AC0A8E0FF1F6D090100510201009901010084
S31500009AD0910101008D0801005AE0FF1F68F4FF1F85
S31500009AE084F00F4000F00F4000A004404C0000201E
S31500009AF0006808B9203423E1F9480088C005C00D84
S31500009B0005D1F7480068400AF649086006E0F448BF
S31500009B100068012101EB5020F2490860A4F1080019
S31500009B20285C5F281BD0A4F10800285C2E2816D0DC
S31500009B30019848B1A4F10800285C5F280FD0A4F171
S31500009B400800285C2E280AD0A4F10800285CE52825
S31500009B5014D1B9F1030F11D0B9F1010F0ED0E248BB
S31500009B600068E2490968884201D10120009000207E
S31500009B70DB490860DB4908602034E1E0DC48007816
S31500009B80012811D1DB48007870B9DB480068D74955
S31500009B900968884208D30420D84908700020FFF7D6
S31500009BA09AFD4FF0FF3099E600200090D2480068F9
S31500009BB078B3D1480068CD49096888425CD2CB4861
S31500009BC00068CD490968401ACD490968081AC5498F
S31500009BD00968884250D30020CA490870C8480078EE
S31500009BE010F0010F04D0C849C848006800F0FAFF19
S31500009BF0BE480068C0490968401A4FEA402BB94878
S31500009C00007810F0010F05D0B64800684008401CE7
S31500009C1003E031E0B348006840080290002622E0E5
S31500009C200BEB8620BA4909684FF480620B69B64986
S31500009C30984720B9FFF7BBFD4FF0FF304EE63046A0
S31500009C4000F09FFF20B9FFF7B2FD4FF0FF3045E669
S31500009C50B002AD4900F0C6FF20B9FFF7A8FD4FF0EE
S31500009C60FF303BE6761C02988642D9D30120FFF7E7
S31500009C7032FD4FF0FF3031E64FF0010A083C01207B
S31500009C80A449087060E0285D612802DB285D7A2817
S31500009C9005DD285D412851DB285D5A284EDC601C15
S31500009CA0285C612803DB601C285C7A280BDD601CBD
S31500009CB0285C412803DB601C285C5A2803DD601CF5
S31500009CC0285C20283AD1A01C285C612803DBA01C54
S31500009CD0285C7A280BDDA01C285C412803DBA01C2D
S31500009CE0285C5A2803DDA01C285C202826D1A4F174
S31500009CF00800285C612804DBA4F10800285C7A28A7
S31500009D0009DDA4F10800285C412817DBA4F108004E
S31500009D10285C5A2812DCA4F10800285C2E280DD0F5
S31500009D20A4F10800285C5F2808D001207349087058
S31500009D300020FFF7D0FC4FF0FF30CFE5203400BF06
S31500009D40761C4645FFF4E5AD00BF009848B166486D
S31500009D500068644909680844634908600020FFF701
S31500009D6087FCBAF1010F01D12046B7E54FF0FF306D
S31500009D70B4E52DE9F04104460D46164666480078DE
S31500009D80022802D15F48007808B9BDE8F08163482F
S31500009D900068002853D0002000F0C6FC4FF4007184
S31500009DA0284605F092FC072C36D25D4800EBC4002D
S31500009DB042685B4850F83410284605F06DFC012CCB
S31500009DC007D15848007820B9FF20A8710F20E87104
S31500009DD022E0032C20D153480078E8B9504901EB22
S31500009DE0C4014968481920224F4905F055FC4F49DE
S31500009DF0424A127851F8220005F072FCC1B2484876
S31500009E0000EBC40040681C3029540421444800EB90
S31500009E10C40040681A302954072C10D14349374AE8
S31500009E20127851F8220005F05BFC07463F48334A9A
S31500009E30127850F822103A46284605F02DFC00BF4D
S31500009E40A3E710B52E48007810F0010F1ED12E4959
S31500009E502E48006800F0C6FE38B92C48006800F5A8
S31500009E6080602A490860012010BD254800681D4908
S31500009E700968884204D10120FFF72DFC0020F3E792
S31500009E802248006800F58060204908601C48006888
S31500009E9014490968884211D11948007810F0010F59
S31500009EA007D019491948006800F09CFE08B901203E
S31500009EB0DAE70120FFF70FFC0020D5E70020D3E703
S31500009EC02DE9F04104460D46174600261248007853
S31500009ED0022802D10B48007808B9BDE8F08127E0D6
S31500009EE078E0FF1F7CE0FF1F54E0FF1FA0E0FF1F8C
S31500009EF09AE0FF1F9BE0FF1F94E0FF1F5AE0FF1F41
S31500009F0080E0FF1F58E0FF1F280C00208CE0FF1F99
S31500009F104C00002099E0FF1FC4E0FF1F84000020D2
S31500009F201CE0FF1F59E0FF1FF30D01005CE0FF1F5F
S31500009F30032C01D0042C3FD1E1B22846FFF79BFC4D
S31500009F400646701C38D08B48007810B901208A4923
S31500009F50087088480078012817D188480068884921
S31500009F600968884211D18748006801280DD18648C2
S31500009F70007840B9012084490870844801684FF48C
S31500009F80805006F057F8BDE8F0817A48007801283D
S31500009F9012D17F4800687F49096888420CD177480A
S31500009FA0006877490968884206D97648006801281A
S31500009FB002D1FFF790FBE6E7042C75D900F0BEFB53
S31500009FC06D48007810B901206A4908707248006827
S31500009FD040B171480068401CA04203D001206F497F
S31500009FE00870D0E76E48007828B96E480068844249
S31500009FF001D96C480460FFF7E1FB012800D1C2E7F4
S3150000A0006048006801284FD100F08EFB6348007855
S3150000A01060B164480068844208D100F0CBFD00B905
S3150000A020B1E700205D4908705F4908705D48006827
S3150000A030A04200D9A7E75A48007870B95948006885
S3150000A040A0420AD1012056490870504801684FF4D1
S3150000A050005005F0EFFF4E4804605148007850B9B3
S3150000A06050480068A04206D00520504908700020DC
S3150000A070FFF731FB87E74A480078012815D14748A2
S3150000A080007890B942480068A0420ED04048006867
S3150000A0903A4909680844A04207D00220434908709B
S3150000A0A00020FFF718FB6EE739E0374800780128F3
S3150000A0B002D10020344908703948007860B1394827
S3150000A0C00068844208D100F075FD00B95BE7002006
S3150000A0D032490870344908702F48046027480068E0
S3150000A0E0401C264908600846007810F0010F01D090
S3150000A0F02F4800E02F4830490860FFF7A2FE0128EC
S3150000A1000DD12E48007830B104202849087000206F
S3150000A110FFF7E1FA37E701202349087033E700BF6C
S3150000A12031E72748007858B90120254908700023EF
S3150000A130244A49F20561AFF63D20DFF88CC000DF06
S3150000A1404FF480202149086040122149086001200F
S3150000A150204908601D4800681D490968B0FBF1F0F8
S3150000A1601D49086013481449086001201B4908600E
S3150000A1707047000084E0FF1F85E0FF1F80E0FF1F9F
S3150000A1807CE0FF1F88E0FF1F98E0FF1FA8E0FF1F8D
S3150000A19094E0FF1FA0E0FF1F9CE0FF1F9BE0FF1F56
S3150000A1A091E0FF1F54E0FF1F9AE0FF1F5AE0FF1FD8
S3150000A1B0280E0020280C0020A000002099E0FF1F98
S3150000A1C0A4E0FF1F28100020D908010090000020FD
S3150000A1D094000020980000209C00002084000020AD
S3150000A1E010B5B04B03EB10131B780B7000F00F0388
S3150000A1F0AC4CE35C137010BD70B503460020002420
S3150000A2001DE01E78302E04DB1E78392E01DC302549
S3150000A2100EE01E78412E04DB1E78462E01DC372523
S3150000A22006E01E78612E03DB1E78662E00DC5725BD
S3150000A2301E7800FB0266701B5B1C661CF4B28C4227
S3150000A240DFDB70BD70B50025242097490870487083
S3150000A25088701820C8702D1D00240AE093480068F5
S3150000A2602430025D2946681CC5B28F484254601CE2
S3150000A270C4B2042CF2DB002409E08D480068025DBC
S3150000A2802846691CCDB288490A54601CC4B2042C05
S3150000A290F3DB002414E0022313FB04535B1C824E01
S3150000A2A09A19022313FB04539919C4F10303DE0020
S3150000A2B0804B1B68F340D8B2FFF792FF601CC4B214
S3150000A2C0042CE8DB05F10800C5B2002414E00223E3
S3150000A2D013FB04535B1C744E9A19022313FB04539D
S3150000A2E09919C4F10303DE00734B1B68F340D8B21F
S3150000A2F0FFF776FF601CC4B2042CE8DB05F108000A
S3150000A300C5B200206849485570BD70B5002666483C
S3150000A310001D05F0E5F9C5B2022000EB45006749CE
S3150000A320087003204870B61C002416E0204604EB93
S3150000A330D0714910B4EB410109D104EBD071491039
S3150000A340091D594A515C32195C4B995403E00020AF
S3150000A35031195A4A5054601CC4B2B4EB450FE5DBC0
S3150000A36006EB4500C6B200205449885570BD4E48DC
S3150000A370704710B54C48001D05F0B2F9022101EBFB
S3150000A3804000C0B210BD4D48704770B51022042180
S3150000A390464800682430FFF72FFF044610220421A8
S3150000A3A043480068FFF728FF054644EA054042494E
S3150000A3B00860084600683F49096848403E49086009
S3150000A3C010220821394800682830FFF715FF064695
S3150000A3D03948006870403849086070BD0022426004
S3150000A3E00160704730B50146002000BF01234C686C
S3150000A3F02CB1334C246824780CB900244C604C688A
S3150000A400F4B90D686C1C0C602878402818D10C68CB
S3150000A4102278412A06D1244C241D294D2C60012482
S3150000A4204C6000E000BF00BF4C684CB10C68641C77
S3150000A4300C60234C2468247814B900244C60002353
S3150000A4404C683CB11E4C246820781D4C2468641C62
S3150000A4501B4D2C60002BC9D030BD7CB5002519489A
S3150000A460007858B9134800F023F9FFF78EFFFFF77D
S3150000A470E9FEFFF74AFF01201249087012496846B3
S3150000A480FFF7ACFF00BF6846FFF7ACFF04462CB1F0
S3150000A49028466D1C00F500700C490C54002CF2D1B6
S3150000A4A001207CBD80100100B81000204C00002067
S3150000A4B0380000204400002048000020D51000206D
S3150000A4C0400000203C000020940F0100280C0020D2
S3150000A4D070B56948806B40F4805067498863881579
S3150000A4E0664908611020664908606649C1F8D400CB
S3150000A4F00846D0F8C80040F01000C1F8C8005E4811
S3150000A500806B40F480505C4988634FF488605B49F7
S3150000A51088615948C06B40F080705749C8635A48F3
S3150000A520406D40F00400584948650846406D20F0EB
S3150000A530010048650846D0F8800020F00100C1F807
S3150000A54080000846406E20F0806048660846406EEF
S3150000A55020F0807048660846006820F020000860F9
S3150000A5600846C06B40F020014748C163C06B40F00D
S3150000A57008014548C163C06B20F004014248C1632D
S3150000A5804FF00000404948604048006805F0F0F888
S3150000A59005464FF08E4105F0ABF8044605F0EDF8A0
S3150000A5A0394988600020C8643848006805F0E0F83A
S3150000A5B006464FF08E4105F09BF8054605F0DDF89E
S3150000A5C0044600EBD47041102F48016408202E4940
S3150000A5D008600846406D20F00400486570BD38B13B
S3150000A5E02B49096841F01001264AC2F8C81006E056
S3150000A5F02849096841F01001224AC2F8C410704780
S3150000A6000020704730B50246234802602348018087
S3150000A6101948806B40F48050174B98632048406877
S3150000A62040F080701E4B58601E485860292000F08C
S3150000A6301F040123A3401C4C450944F8253000BFE4
S3150000A64000BF00F01F040123A34044094FF0E0259A
S3150000A65005EB8404C4F8003100BF30BD1348006820
S3150000A660022808D10E48406840F080700C494860C6
S3150000A67040F21310486070470080044000C0044058
S3150000A680C0F00F4000F00F400080034000000020A3
S3150000A690C8F00F40C4F00F40B0E0FF1FACE0FF1F52
S3150000A6A000A0044013010A0080E200E0A0A00440DC
S3150000A6B00649096E054AD26D5140044A926D5140D1
S3150000A6C0024A526D5140016070470000008004400C
S3150000A6D000240320DFF850C300DF17E0DFF84CC387
S3150000A6E000DFD34801680220DFF848C300DF2046B8
S3150000A6F0611CCCB2032190FBF1F201FB120028B9D8
S3150000A700CB4801680120DFF82CC300DFE6E710B56F
S3150000A710044614B10120C8490860C54801680420F0
S3150000A720DFF810C300DF10BD0121C44A116008B173
S3150000A730022100E00121C24A11707047BC4801683D
S3150000A7401020DFF8F0C200DF7047B94801684FF407
S3150000A7500070DFF8E0C200DF7047B548016880206E
S3150000A760DFF8D0C200DF7047B14801684FF480704F
S3150000A770DFF8C0C200DF704708E0AF48006828B9BC
S3150000A78002F030FF02F079FF02F05FFFF5E71CB53B
S3150000A7904FF0000ADFF8ACC200DFA5490860FFF7FA
S3150000A7A097FE03F021F800F081F90120FFF717FF6B
S3150000A7B004219F480068FFF725FF4FF0010B00209A
S3150000A7C003F01DF80026B04601209F4908700225B7
S3150000A7D00027002099490860FFF73FFE00239B4AA7
S3150000A7E044F20B61AFF21710DFF864C200DF4FF0DE
S3150000A7F001099848006841680320884704F0ECFE88
S3150000A80004F0FCFE02E100224FF6FF7140F2F73041
S3150000A810DFF844C200DFDFF844C200DF044614F468
S3150000A820007F04D00026042506208749087014F00E
S3150000A830100F05D04FF00A08012601207F49086055
S3150000A84014F0200F02D004207F49087014F0040F82
S3150000A8502AD000207A490870FFF7C1FEFEF714FCE3
S3150000A8607548006890B17B480068416800208847B9
S3150000A870FFF77DFD0190019804F032FF014600903C
S3150000A880019802F0CAFE00206B4908607148006812
S3150000A8904168022088474FF0010901206849087085
S3150000A8A0FFF79DFE4FF0000B14F0800F0ED004F062
S3150000A8B0BEFE68480068416804208847002002F010
S3150000A8C09EFF0020FFF78BFE00BFFEE714F4807F9B
S3150000A8D006D004F0ACFE5F48006841680420884753
S3150000A8E014F0010F76D0BBF1000F06D104215048B9
S3150000A8F00068FFF787FE4FF0010BB9F1000F05D096
S3150000A900B9F1030F03D14FF0000901E000E000BFE9
S3150000A91000BF6EB1012E0AD1B8F1000F03D0A8F125
S3150000A9200100804600E0002000B9002601E000BFDB
S3150000A93000BF00BF44480078072847D2DFE800F090
S3150000A940481C472946040C002EB9002002F057FF88
S3150000A95000203D4908703CE06EB915B1681E0546F9
S3150000A96000E0002038B9002002F049FF01203649F6
S3150000A9700870FFF772FD2CE015B1681E054600E071
S3150000A980002028B9012002F03AFF03202E49087062
S3150000A9901FE002F04DFFB8B1BAF1000F11D100234C
S3150000A9A02F4A30493048DFF8A8C000DF00232F4A7D
S3150000A9B049F20161AFF23F20DFF894C000DF4FF0AB
S3150000A9C0010A02202049087003E003E000BF00BF2F
S3150000A9D000BF00BF14F0020F18D018480068A8B1D5
S3150000A9E017480078012803D01548007802280DD1B1
S3150000A9F00FB1002707E0012711480078012802D18E
S3150000AA0000200E4908603846FFF7E9FDFBE610B561
S3150000AA10FDF706FD164A4BF20A41AFF28D20DFF82C
S3150000AA2054C000DF002010BD6D0301008503010046
S3150000AA30BCE0FF1FF1010100B4E0FF1FC0E0FF1FF3
S3150000AA40B8E0FF1F6D090100C4E0FF1F10110020D0
S3150000AA50D90801004C0000205102010099010100B3
S3150000AA60501100200F5E010013960000A81200206E
S3150000AA7038130020F906010003460022B3F5806F63
S3150000AA8012D100BF06E0885CFF2801D00020704785
S3150000AA90501C82B20C2AF6DB887BFF2802D1C87BC9
S3150000AAA0FF2801D00020F2E70120F0E710B501F001
S3150000AAB02BFC00BF2020654908604FF04000644928
S3150000AAC0C1F884004FF0010088644FF010008860E0
S3150000AAD04FF0020048640846406940F010004861A3
S3150000AAE00846806840F0100088600846806C40F098
S3150000AAF0010088644FF0020048640846406D40F04B
S3150000AB000200486540F213105249486000BF4FF0FA
S3150000AB10010010BD20B100214F4A116000BF04E0C2
S3150000AB2001214D4A116000BF00BF70471CB54B4C58
S3150000AB302468E469A26B494C2468E469E16B474CDC
S3150000AB402468E469606B454C24686369984708B9D2
S3150000AB5000201CBD00200090404A01901268D26976
S3150000AB6011683E4A1268D26902F120003B4A126817
S3150000AB70002394691A46A04708B90020E9E7012096
S3150000AB80E7E77CB5044600200090A202334B019013
S3150000AB901B68DB695969314B1B68DB6903F12000CF
S3150000ABA02E4B1B689D690023A84708B900207CBD71
S3150000ABB00120FCE71CB500200090284A019012688D
S3150000ABC0D2691169254A1268D26902F12000234A26
S3150000ABD01268002394691A46A04708B900201CBDD4
S3150000ABE00120FCE77CB504460D4629462046FFF7C2
S3150000ABF043FF08B900207CBD18490968C969086B7C
S3150000AC00164909684FF480624B692946984708B986
S3150000AC100020F0E7002111480068C069006B0F4A68
S3150000AC20CDE900011268D26991690C4A1268D269AD
S3150000AC3002F12000094A12684FF4806396692246A1
S3150000AC40B04708B90020D6E70120D4E784F00F40CA
S3150000AC5000F00F4000A004400408FE434C00002012
S3150000AC602020F84908604FF04000F749C1F88400F9
S3150000AC704FF0010088644FF0100088604FF002002A
S3150000AC8048640846406940F01000486108468068FC
S3150000AC9040F0100088600846806C40F0010088642F
S3150000ACA04FF0020048640846406D40F002004865D7
S3150000ACB040F21310E5494860704710B503460C464C
S3150000ACC000210020014606E0C80024FA00F058548E
S3150000ACD0481CC0B201469142F6DB10BD2DE9F04199
S3150000ACE006460F4600250BE03946304602F0E7FAE5
S3150000ACF00446022C02D02046BDE8F081681CC5B28D
S3150000AD000A2DF1DB2046F7E7F8B504460D4604F0B8
S3150000AD100C0040F0020669463046FFF7DFFF0746A3
S3150000AD209DF8030000069DF8021040EA01409DF8D8
S3150000AD30011040EA01209DF8001008432860012F09
S3150000AD4001D10120F8BD0020FCE7F8B504460D4608
S3150000AD50082C08D1BE480068A84201D10120F8BDE0
S3150000AD60BB48056000E000BF00BF04F00C060422EB
S3150000AD7029466846FFF7A1FF69463046FFF7AEFF52
S3150000AD800746012F00D1EAE70020E8E72DE9F8435E
S3150000AD9004460E4604F07F4804F0F00948EA09012B
S3150000ADA00820FFF7D2FF10B90020BDE8F88304F0B1
S3150000ADB00C0040F0030769463846FFF78FFF6946E7
S3150000ADC03846FFF78BFF05469DF8030000069DF801
S3150000ADD0021040EA01409DF8011040EA01209DF86A
S3150000ADE0001008433060012D01D10120DDE700206D
S3150000ADF0DBE72DE9F84304460D4604F07F4804F0EE
S3150000AE00F00948EA09010820FFF79FFF10B9002062
S3150000AE10BDE8F88344B98E484068A84201D10120B4
S3150000AE20F6E78B48456000E000BF00BF04F00C0069
S3150000AE3040F00107042229466846FFF73EFF6946AF
S3150000AE403846FFF74BFF012801D00020E0E70E2728
S3150000AE5000213846FFF742FF0646012E00D1D7E70C
S3150000AE600020D5E72DE9F84F07468846144614B961
S3150000AE700020BDE8F88F4FEA940A76490020FFF7D4
S3150000AE80B8FF08B90020F4E74FF005090422394657
S3150000AE906846FFF712FF69464846FFF71FFF01287D
S3150000AEA001D00020E5E74FF00D0900250AE04146F4
S3150000AEB04846FFF713FF012801D00020D9E708F123
S3150000AEC004086D1C5545F2D34FF00E090021484683
S3150000AED0FFF704FF0646012E00D1CAE70020C8E7A7
S3150000AEE02DE9F84F07468846144614B90020BDE8F8
S3150000AEF0F88F4FEA940A57490020FFF77AFF08B9FE
S3150000AF000020F4E74FF00509042239466846FFF7AA
S3150000AF10D4FE69464846FFF7E1FE012801D000202D
S3150000AF20E5E74FF00F0941464846FFF7D7FE0128EF
S3150000AF3001D00020DBE700260AE041464846FFF73D
S3150000AF40CDFE012801D00020D1E708F10408761CC7
S3150000AF505645F2D34FF00E0900214846FFF7BEFED4
S3150000AF600546012D00D1C2E70020C0E72DE9FC41CE
S3150000AF7005460E460422294601A8FFF79EFE052730
S3150000AF8001A93846FFF7AAFE012802D00020BDE835
S3150000AF90FC810F2769463846FFF7A0FE012801D03D
S3150000AFA00020F4E70E2769463846FFF797FE044669
S3150000AFB09DF8030000069DF8021040EA01409DF846
S3150000AFC0011040EA01209DF8001008433060012C72
S3150000AFD001D10120DBE70020D9E7F8B505460E468A
S3150000AFE0042229466846FFF768FE05276946384663
S3150000AFF0FFF774FE012801D00020F8BD0422314677
S3150000B0006846FFF75AFE0D2769463846FFF766FE83
S3150000B010012801D00020F0E70E2700213846FFF76F
S3150000B0205DFE0446012C00D1E7E70020E5E770B598
S3150000B03004460D4607490020FFF7DBFE60B90020F5
S3150000B04070BD000084F00F4000F00F4000A00440E7
S3150000B050500000205200002329462046FFF786FFB5
S3150000B06008B90020ECE70120EAE770B504460D4672
S3150000B070FE490020FFF7BDFE08B9002070BD294635
S3150000B0802046FFF7AAFF08B90020F7E70120F5E7F9
S3150000B09038B504460D46F549891E0020FFF7A9FE7E
S3150000B0A008B9002038BD69462046FFF75FFF08B99A
S3150000B0B00020F7E7A007C10E0098C84028700120BD
S3150000B0C0F0E770B504460E46E849891E0020FFF7F2
S3150000B0D090FE08B9002070BDA007C00E06FA00F564
S3150000B0E029462046FFF779FF08B90020F3E701203B
S3150000B0F0F1E72DE9F04105460F4614460AE03946C8
S3150000B1002846FFF7C5FF10B90020BDE8F0816D1C89
S3150000B1107F1C641E14B115F0030FF0D117E0D4485C
S3150000B1200068016AD2480068006A401E28400E1A6C
S3150000B130B44201D224F00306324639462846FFF7C8
S3150000B140CFFE08B90020E0E735443744A41B032CA2
S3150000B150E5D809E039462846FFF79AFF08B90020E6
S3150000B160D3E76D1C7F1C641E002CF3D10120CCE7B5
S3150000B1702DE9F04105460E4614460AE03178284688
S3150000B180FFF79FFF10B90020BDE8F0816D1C761C0B
S3150000B190641E14B115F0030FF0D117E0B44800682F
S3150000B1A0016AB3480068006A401E28400F1ABC4274
S3150000B1B001D224F003073A4631462846FFF752FEED
S3150000B1C008B90020E0E73D443E44E41B032CE5D8E3
S3150000B1D009E031782846FFF774FF08B90020D3E765
S3150000B1E06D1C761C641E002CF3D10120CCE773B5D0
S3150000B1F00446002564269F480199FFF736FF08B9E3
S3150000B20000207CBD44F480319A48001FFFF72DFFD3
S3150000B21008B90020F5E700250EE001A99548083891
S3150000B220FFF705FF08B90020EBE7019810F4803F0F
S3150000B23001D00120E5E76D1CB542EEDB0020E0E71A
S3150000B24038B5054600210820FFF77FFD08B9002024
S3150000B25038BD002408E055F824102046FFF7C7FF44
S3150000B26008B90020F4E7641C042CF4D30920696AA9
S3150000B270FFF7BDFF08B90020EAE70D2408E055F8FE
S3150000B28024102046FFF7B3FF08B90020E0E7641C4E
S3150000B290102CF4D31020296CFFF7A9FF08B9002061
S3150000B2A0D6E7754973480838FFF7DFFE08B900206E
S3150000B2B0CEE769460420FFF727FD08B90020C7E757
S3150000B2C0009810F0A00F01D00020C1E70120BFE7D1
S3150000B2D02DE9F04105460E460024642729466548B7
S3150000B2E0001FFFF7C2FE10B90020BDE8F081002460
S3150000B2F00DE031465F480838FFF799FE08B900208F
S3150000B300F3E7306810F4803F00D002E0641CBC42D2
S3150000B310EFDB00BFBC4201D10020E6E731465548CD
S3150000B320FFF785FE08B90020DFE70120DDE73EB51F
S3150000B330044600210820FFF708FD08B900203EBD9D
S3150000B34001A90020FFF7C4FF08B90020F7E79DF820
S3150000B350070000069DF8061040EA01409DF805101A
S3150000B36040EA01209DF80410084320606946042045
S3150000B370FFF7CAFC08B90020E1E7009810F0A00F1B
S3150000B38001D00020DBE70120D9E738B504460D4699
S3150000B390694638480838FFF74AFE08B9002038BD24
S3150000B3A0009810F4003F01D10020F8E72146002064
S3150000B3B0FFF78EFF08B90020F1E729460120FFF7C5
S3150000B3C087FF08B90020EAE70120E8E738B542F22E
S3150000B3D0107500240EE0694626480838FFF727FE58
S3150000B3E008B9002038BD009810F4003F01D00120B4
S3150000B3F0F8E7641CAC42EED30020F3E738B5044608
S3150000B40021460020FFF7F3FE08B9002038BD694643
S3150000B4100F20FFF75DFF08B90020F7E70099891CA8
S3150000B4200F20FFF7E4FE08B90020EFE712491148A4
S3150000B4300838FFF71AFE08B90020E7E70120E5E71C
S3150000B4402DE9F04391B004460D4616461F46DDE948
S3150000B45018894FF08070109000960197CDF80880FB
S3150000B460CDF80C9000200490059007E052000023D0
S3150000B4704C000020F8ED00E001005FA00690079068
S3150000B4800890A068099000200A900B900C90E06844
S3150000B4900D9060680E900F956846FFF7D1FE18B9BB
S3150000B4A0002011B0BDE8F083FFF790FF08B9002037
S3150000B4B0F7E76846FFF73BFF08B90020F1E7009879
S3150000B4C008B10020EDE70120EBE71CB5002400BF22
S3150000B4D004E0FF200DF80400601CC4B2082CF8DB61
S3150000B4E06946332000F09CFF01201CBD38B5044698
S3150000B4F0E0B28DF80000200A8DF8010069461020A0
S3150000B50000F08EFF012038BD1CB5044600200190D6
S3150000B51001A9082000F084FF69460020FFF7F4FB2C
S3150000B520012801D000201CBD9DF8030000069DF8EF
S3150000B530021040EA01409DF8011040EA01209DF802
S3150000B5400010084320600120EDE710B5C649C74842
S3150000B550FFF78BFD08B9002010BD0120FCE708B5F8
S3150000B5606946C348FFF712FC08B9002008BD0098D9
S3150000B570A0F5E011203901D00020F7E76946BC4864
S3150000B580F838FFF703FC08B90020EFE769464FF0EB
S3150000B5908070FFF7FBFB08B90020E7E7009810F082
S3150000B5A0040F3AD0B348006841680020884714E089
S3150000B5B00121AF48F838FFF71CFC08B90020D5E791
S3150000B5C069464FF08070FFF7E1FB08B90020CDE730
S3150000B5D0009810F0010F00D000E0E9E700BF1AE084
S3150000B5E00021A348F838FFF704FC08B90020BDE79E
S3150000B5F069464FF08070FFF7C9FB08B90020B5E730
S3150000B60069469B48F838FFF7C1FB08B90020ADE74B
S3150000B610009800B900E0E3E700BF0120A6E708B5FF
S3150000B62000200090FFF751FF08B9002008BD4EF238
S3150000B6309E70FFF75BFF08B90020F7E7FFF745FFAD
S3150000B64008B90020F2E76846FFF75EFF08B9002058
S3150000B650ECE70120EAE708B500200090401E864985
S3150000B6600860486000F050FEFFF7FAFA0120FFF785
S3150000B67051FAFFF7D4FF08B9002008BD1E210020AB
S3150000B680FFF763FB08B90020F7E700210820FFF762
S3150000B6905CFB08B90020F0E74FF0A0410420FFF75B
S3150000B6A054FB08B90020E8E700BF69460420FFF70D
S3150000B6B02BFB08B90020E0E7009800F02040B0F12D
S3150000B6C0204FF2D16D490420FFF73FFB08B9002057
S3150000B6D0D3E7FFF744FF00210820FFF736FB08B940
S3150000B6E00020CAE70120C8E738B50446062C7AD2FE
S3150000B6F0DFE804F003400716878D0120FFF70AFAFA
S3150000B700AFE00120FFF706FA0220DFF874C100DF80
S3150000B7100020FFF7FFF90220DFF864C100DFA0E098
S3150000B7200120FFF7F7F90120DFF854C100DF002000
S3150000B730FFF7F0F90120DFF848C100DFFFF78BFFC4
S3150000B74008B9002038BD4849491C4848FFF78DFC18
S3150000B75008B90020F6E70120FFF7DCF90120DFF841
S3150000B76020C100DF0020FFF7D5F90120DFF810C166
S3150000B77000DF76E00120FFF7CDF90220DFF800C1F7
S3150000B78000DF0020FFF7C6F90220DFF8F4C000DF73
S3150000B790FFF761FF08B90020D4E73349491C334855
S3150000B7A0FFF763FC08B90020CCE701212F480C30D5
S3150000B7B0FFF75BFC08B90020C4E70120FFF7AAF9F0
S3150000B7C00220DFF8BCC000DF0020FFF7A3F902204B
S3150000B7D0DFF8ACC000DF00BF69462448FFF727FC4E
S3150000B7E010B90020AEE73AE0009810F4003FF3D01D
S3150000B7F000211E480C30FFF738FC08B90020A1E7ED
S3150000B8002FE0FFF7A2FE08B900209BE729E000F031
S3150000B8107BFDFFF725FAFFF702FF08B9002091E745
S3150000B8201E210020FFF791FA08B900208AE70021BF
S3150000B8300820FFF78AFA08B9002083E74FF0A041F5
S3150000B8400420FFF782FA08B900207BE70649491C65
S3150000B8500648FFF70AFC08B9002073E701E000205C
S3150000B86070E700BF01206DE700005FA0F0ED00E08B
S3150000B870FC0000014C00002050000020000F00508A
S3150000B8809101010002460020052A1AD008DC012A8F
S3150000B8900FD0022A0ED0032A0DD0042A21D10BE0A4
S3150000B8A0062A0FD0F02A0ED0FE2A16D0FF2A18D16B
S3150000B8B00DE016E015E014E0F74B1B680B60042062
S3150000B8C00FE00EE00DE001230B70012009E040239C
S3150000B8D00B7000234B70022003E005230B70012040
S3150000B8E000BF00BF70474FF47A51484301460A46ED
S3150000B8F000BF00BF531E1A00FCD100BF704730B511
S3150000B90002460B461078547840EA0421090108469D
S3150000B910044600BF00BF651E2C00FCD100BF0020FE
S3150000B9201870012030BD10B50246107810B10128FC
S3150000B9300DD107E0537803F00100C343D74C2360D1
S3150000B94000BF08E0537803F0010000BF03E0FF20CA
S3150000B9500870012010BD00BF002008700120F9E723
S3150000B96070B506460D46307808B9012400E03478F3
S3150000B97003F05DFE012C31D10120C949087000BFDA
S3150000B9802020C84908604FF04000C749C1F884002C
S3150000B9904FF0010088644FF0100088604FF00200FD
S3150000B9A048640846406940F01000486108468068CF
S3150000B9B040F0100088600846806C40F00100886402
S3150000B9C04FF0020048640846406D40F002004865AA
S3150000B9D040F21310B549486000BF03E0002028700C
S3150000B9E0012070BD00BF2C700120FAE710B5044697
S3150000B9F00020AB49087000BF0120AB494864102005
S3150000BA004860022048640846806C40F02000A8493F
S3150000BA100860A648406840F08070A4494860A54880
S3150000BA20486000BF03F0EAFD00202070012010BD31
S3150000BA30014600BF0020487008700220704770B5AC
S3150000BA4003460D4619785A789878DE7840EA06203B
S3150000BA501E7940EA06405E7940EA066412F0010F5C
S3150000BA600ED011F0010F05D000BF20208D4E3060A2
S3150000BA7000BF05E000BF20208D4E306000BF00BF34
S3150000BA8012F0020F0ED011F0020F05D000BF4020B9
S3150000BA90844E306000BF05E000BF4020844E306019
S3150000BAA000BF00BF12F0040F02D0880800BF00BF1D
S3150000BAB012F0200F02D0480900BF00BF12F0800F1D
S3150000BAC004D0C8097C4E306000BF00BF002C57D0A0
S3150000BAD07A48844200D9044600BF00204FF0E02691
S3150000BAE0B06177486043774EB0FBF6F04FF0E02642
S3150000BAF070610520306100BF00BF12F0010F04D055
S3150000BB0000BF0020484000D02AE012F0020F08D003
S3150000BB1000BF6D480068C0F3C01090EA510000D025
S3150000BB201EE012F0040F05D000BF002090EA91003D
S3150000BB3000D015E012F0200F05D000BF002090EADB
S3150000BB40511000D00CE012F0800F08D000BF56480C
S3150000BB50006DC0F3400090EAD11000D000E007E08D
S3150000BB6000BF4FF0E0200069C0F300400028C4D0B9
S3150000BB7000BF00BF00204FF0E026306100BF00BFCD
S3150000BB8000BF002600BF50480068C0F3C01046EA58
S3150000BB90400000BF40EA860000BF40EAC60000BF82
S3150000BBA040EA46164048006DC0F3400046EAC01120
S3150000BBB029704FF0010070BD30B502460C46107872
S3150000BBC0557840EA0520957840EA0540D57840EA60
S3150000BBD005631BB9FF202070012030BD3B4883421E
S3150000BBE004D301202E4D6870686012E000202C4DB1
S3150000BBF06870581E364D2844B0FBF3F1022905D96A
S3150000BC00891E881C0325B0FBF5F100E001212448BC
S3150000BC104160002020700120DFE770B504460D4624
S3150000BC2014F8016B0EB94FF480762146304600F0C9
S3150000BC30F7FB00202870012070BD10B5024613786E
S3150000BC4003F00300401C164C2075C3F3800414480F
S3150000BC50447500200870012010BD38B504460D4615
S3150000BC600F480078012803D0FF202870012038BD36
S3150000BC706078A17840EA0120E17840EA0140217924
S3150000BC8040EA016000906946002001F018FB0020A0
S3150000BC9028700120EBE70000F81601001018FE439B
S3150000BCA068F4FF1F84F00F4000F00F4000A004402E
S3150000BCB088F00F4013010A000408FE43C0C62D0099
S3150000BCC0006CDC0240420F0090F00F40001BB700F2
S3150000BCD000366E0102461078FE4B18725078937843
S3150000BCE040EA0323FB484381D078137940EA0323D3
S3150000BCF0F848838100200870012070472DE9F04F35
S3150000BD0085B006460C46002003900025A146A41CDB
S3150000BD10F149087082460290761C16F8010B0490D1
S3150000BD203AE116F8018B18F0020F7CD0BAF1000F39
S3150000BD303AD0E848478908F01100012810D100BF21
S3150000BD406946404601F0BBFA0546022D1AD1380075
S3150000BD50A7F1010716D0E04800780028F0D011E0DE
S3150000BD6000BF69460E2001F0AAFA0546022D07D14A
S3150000BD703800A7F1010703D0D74800780028F0D093
S3150000BD804FF0000A012D00D00CE1009804F8010BD9
S3150000BD900098000A04F8010B0098000C04F8010B47
S3150000BDA00098000E04F8010B18F0100F56D03078EA
S3150000BDB0717840EA0120B17840EA0140F17840EA22
S3150000BDC0016B361DC3488089019018F0010F14D00D
S3150000BDD0C048478900BF0021404601F070FA054679
S3150000BDE0022D07D13800A7F1010703D0BA48007821
S3150000BDF00028F0D0012D00D0D4E000BFB548478917
S3150000BE0000BF6946404601F05AFA0546022D07D1A1
S3150000BE103800A7F1010703D0AF4800780028F0D01A
S3150000BE20012D01D00EE05CE0AA48006900990840A7
S3150000BE30584507D00198411E019118B1A6480078CF
S3150000BE400028DBD000BFA348006900990840584588
S3150000BE5001D045F01005012D40D0A3E09D4847894B
S3150000BE6018F0010F18D0BAF1000F37D100BF00212A
S3150000BE70404601F024FA0546022D07D13800A7F105
S3150000BE80010703D0944800780028F0D0012D00D097
S3150000BE9088E04FF0010A21E000BF6946404601F004
S3150000BEA00EFA0546022D07D13800A7F1010703D087
S3150000BEB0894800780028F0D0012D00D072E0009863
S3150000BEC004F8010B0098000A04F8010B0098000C16
S3150000BED004F8010B0098000E04F8010B00200290F4
S3150000BEE053E0BAF1000F25D07A48478900BF69466A
S3150000BEF00E2001F0E4F90546022D07D13800A7F11E
S3150000BF00010703D0744800780028F0D0012D00D036
S3150000BF1048E0009804F8010B0098000A04F8010BA9
S3150000BF200098000C04F8010B0098000E04F8010BB1
S3150000BF304FF0000A3078717840EA0120B17840EA83
S3150000BF400140F17840EA01600090361D18F0200F9C
S3150000BF5004D0604800990161012516E05D484789D3
S3150000BF6000BF6946404601F0AAF90546022D07D1F1
S3150000BF703800A7F1010703D0574800780028F0D011
S3150000BF80012D00D00EE0012002900398401C039082
S3150000BF905148007800B105E00498411E049100283C
S3150000BFA07FF4BFAE00BF012D3BD1BAF1000F24D004
S3150000BFB04848478900BF69460E2001F080F90546CA
S3150000BFC0022D07D13800A7F1010703D042480078B7
S3150000BFD00028F0D0012D00D024E0009804F8010BD1
S3150000BFE00098000A04F8010B0098000C04F8010BF5
S3150000BFF00098000E04F8010B13E0029888B135484A
S3150000C000478900BF00210E2001F059F90546022D8F
S3150000C01007D13800A7F1010703D02F480078002880
S3150000C020F0D000BF039889F8000089F80150A4EB0E
S3150000C030090005B0BDE8F08F2DE9F84F04460D461E
S3150000C0404FF0000B0026A846ED1C00202249087080
S3150000C050641C2078617840EA012AA41CBAF1000F1A
S3150000C06000D199E014F8017B17F0020F54D017F0B5
S3150000C070010F16D01748B0F80A9000BF00213846C5
S3150000C08001F01DF90646022E08D15FEA0900A9F162
S3150000C090010903D0104800780028EFD0012E00D007
S3150000C0A07AE033E0BAF1000F03D117F0010F00D0A8
S3150000C0B00E270848B0F80A9000BF6946384601F0D6
S3150000C0C0FEF80646022E0DD15FEA0900A9F1010924
S3150000C0D008D003E068F4FF1F58000020C548007828
S3150000C0E00028EAD0012E00D056E0009805F8010B92
S3150000C0F00098000A05F8010B0098000C05F8010BE2
S3150000C1000098000E05F8010B0BF1010B5FEA0A001F
S3150000C110AAF1010AC6D13EE024E02078617840EA1F
S3150000C1200120A17840EA0140E17840EA01600090F0
S3150000C130241DB148B0F80A9000BF6946384601F0A0
S3150000C140BEF80646022E08D15FEA0900A9F10109E8
S3150000C15003D0A84800780028EFD0012E00D01BE0BD
S3150000C1600BF1010B5FEA0A00AAF1010AD5D1A24838
S3150000C170B0F80A9000BF00210E2001F0A0F8064694
S3150000C180022E08D15FEA0900A9F1010903D09948F6
S3150000C19000780028EFD000BF88F800B04FEA1B20D7
S3150000C1A088F8010088F80260A5EB0800BDE8F88F62
S3150000C1B00246FF2008700120704770B506460D46FE
S3150000C1C03078802807DB30789F2804DC2946304603
S3150000C1D0FCF7D2FF70BD307805F8010B16F8010B9D
S3150000C1E0172870D2DFE800F00C141A204E54658828
S3150000C1F078252B888888888830363C4248494A000A
S3150000C2003078691CFFF73EFB04462C70A01CE1E762
S3150000C21029463046FFF787FB044672E0294630463A
S3150000C220FFF79EFB04466CE02846FFF7DFFB04465B
S3150000C23067E029463046FFF762FB044661E0284680
S3150000C240FFF7F6FB04465CE029463046FFF7F7FBAE
S3150000C250044656E029463046FFF7AEFC044650E059
S3150000C26029463046FFF7D9FC04464AE029463046BF
S3150000C270FFF7E3FC044644E000BF00BFFF20287040
S3150000C2800220A7E729463046FFF724FD044638E09A
S3150000C29059480078012805D129463046FFF72EFD7A
S3150000C2A0044604E0002028706870022400BF00BF26
S3150000C2B027E051480078012806D129463046FFF785
S3150000C2C0BBFE044606E017E0002028706870A870E0
S3150000C2D0032400BF00BF14E047480078012805D1B9
S3150000C2E029463046FFF7B9FC044603E0FF202870D4
S3150000C2F002206FE700BF04E0FF2005F8010C0120D3
S3150000C30068E700BF601C65E710B500203A49087071
S3150000C3100220486064213848418101203649087569
S3150000C32000F001F810BD3548806B40F4F0503349F9
S3150000C33088638815324948612020324908603248AE
S3150000C340D0F8940040F02000304908604FF4807027
S3150000C3502B4988614FF040002B49C1F884000846FC
S3150000C360D0F8940040F040002849086040F20310DD
S3150000C3702349C8612448D0F8940020F0800023495E
S3150000C38008604FF48070224908604FF001001E4992
S3150000C39048640846406D40F0010048654FF48070DF
S3150000C3A01C4908614FF0100017494860084640696B
S3150000C3B040F01000486140F22310154948604FF0E4
S3150000C3C00200114948640846406D40F00200486585
S3150000C3D04FF49070104908614FF010000A49C1F8F7
S3150000C3E0C8000846D0F8D40040F010000B49086099
S3150000C3F0704700005800002068F4FF1F00800440CA
S3150000C40000B0044084F00F4000F00F4094F00F405D
S3150000C41000A004400090044000C00440D4F00F4047
S3150000C42070B50022002333E013B911F8012B08235D
S3150000C43012F0010F05D000BF4024FE4D2C6000BF56
S3150000C44005E000BF4024FC4D2C6000BF00BF00BFCC
S3150000C4504FF02004F84D2C6000BFF84D6C6825465F
S3150000C46000BF00BFA5F101063500FBD100BF00BF2C
S3150000C4702024F04D2C6000BFF04D6C68254600BFAF
S3150000C48000BFA5F101063500FBD100BF52085B1EB7
S3150000C4900400A0F10100C7D170BDF0B503460F46F8
S3150000C4A000240120DFF898C3CCF8180000BF00BFB5
S3150000C4B02020DFF880C3ACF1840CCCF8880000BFE4
S3150000C4C000BF00BF00BFCCF8840000BF00BF00BFA4
S3150000C4D01A461346DA48836100BF00BF2020CCF815
S3150000C4E0880000BF00BF00BF00BFCCF8840000BFBB
S3150000C4F000BF00BF14445A081046DFF844C3CCF806
S3150000C500180000BF00BF2020DFF828C3ACF1840C60
S3150000C510CCF8880000BF00BF00BF00BFCCF8840085
S3150000C52000BF00BF00BF14449A081046DFF810C3CE
S3150000C530CCF8180000BF00BF2020DFF8F8C2ACF12D
S3150000C540840CCCF8880000BF00BF00BF00BFCCF849
S3150000C550840000BF00BF00BF1444DA081046DFF8AD
S3150000C560E0C2CCF8180000BF00BF2020DFF8C4C22C
S3150000C570ACF1840CCCF8880000BF00BF00BF00BF40
S3150000C580CCF8840000BF00BF00BF14442046DFF88B
S3150000C590B0C2CCF8180000BF00BF2020DFF894C25C
S3150000C5A0ACF1840CCCF8880000BF00BF00BF00BF10
S3150000C5B0CCF8840000BF00BF00BF0020DFF880C2B7
S3150000C5C0CCF8180000BF00BF2020DFF868C2ACF12D
S3150000C5D0840CCCF8880000BF00BF00BF00BFCCF8B9
S3150000C5E0840000BF00BF00BF0120DFF854C2CCF8B2
S3150000C5F0180000BF00BF2020DFF838C2ACF1840C61
S3150000C600CCF8880000BF00BF00BF00BFCCF8840094
S3150000C61000BF00BF00BF00BF0120CCF8440000BF30
S3150000C6208648017D11E000BF2020DFF808C2ACF18A
S3150000C630840CCCF8880000BF00BF00BF00BFCCF858
S3150000C640840000BF00BF00BF491E0029EBD100BF18
S3150000C6502020DFF8E0C1ACF1840CCCF8880000BFE4
S3150000C66000BF00BF00BF77480068024600BF4FF01A
S3150000C6702000CCF8840000BF00BF00BF164600BFF4
S3150000C680CCF8880000BF00BF00BF00BF6C48D0F8E0
S3150000C6901C02024600BF4FF02000CCF8840000BF09
S3150000C6A000BF00BF46EA420600BFCCF8880000BFC4
S3150000C6B000BF00BF00BF63480068024600BF4FF0DE
S3150000C6C02000CCF8840000BF00BF00BF46EA820607
S3150000C6D0012E7DD113F0020F5ED00025002420210B
S3150000C6E01DE000BF2020DFF84CC1ACF1840CCCF873
S3150000C6F0880000BF00BF00BF00BF52480068024666
S3150000C70000BF4FF02000CCF8840000BF00BF00BF80
S3150000C71014444FEA550545EAC275A1F10101002905
S3150000C720DFD100BF4FF02000DFF81CC1CCF8880035
S3150000C73000BF00BF00BF00BF42480068024600BFFE
S3150000C7404FF02000CCF8840000BF00BF00BF84EA91
S3150000C750020010F0010F00D0082607B13D603748EF
S3150000C760017D0FE000BF2020DFF8DCC0CCF8880098
S3150000C77000BF00BF00BF00BFCCF8840000BF00BFF1
S3150000C78000BF491E0029EDD100BF0120DFF8B8C067
S3150000C790CCF8480000BF5CE02848017D0FE000BFF0
S3150000C7A02020DFF8A4C0CCF8880000BF00BF00BF7F
S3150000C7B000BFCCF8840000BF00BF00BF491E00299F
S3150000C7C0EDD100BF0120DFF880C0CCF8480000E0C2
S3150000C7D063E000BF3D680024202117E02846DFF80B
S3150000C7E060C0CCF8180000BF00BF2020DFF858C09A
S3150000C7F0CCF8880000BF00BF00BF00BFCCF88400A3
S3150000C80000BF00BF00BF2C446D08491E0029E5D1BA
S3150000C81000BF0B48846100BF00BF2020DFF828C09E
S3150000C820CCF8880000BF00BF00BF00BFCCF8840072
S3150000C83000BF0BE084F00F4088F00F4068F4FF1F44
S3150000C8400010FE431C12FE4300F00F4000BF00BF65
S3150000C85000BFFE48017AC1B10020DFF8F4C3CCF86E
S3150000C860180000BF0FE000BF2020DFF8E8C3CCF8B7
S3150000C870880000BF00BF00BF00BFCCF8840000BF27
S3150000C88000BF00BF491E0029EDD10120DFF8C0C35B
S3150000C890CCF8180000BFF0B2F0BD022E01D0042E75
S3150000C8A05DD1EA48407DB0B113F0020F13D02121CB
S3150000C8B00FE000BF2020DFF89CC3CCF8880000BF43
S3150000C8C000BF00BF00BFCCF8840000BF00BF00BFA0
S3150000C8D0491E0029EDD1DD48017D0FE000BF202073
S3150000C8E0DFF870C3CCF8880000BF00BF00BF00BFF0
S3150000C8F0CCF8840000BF00BF00BF491E0029EDD15F
S3150000C90000BF0120DFF84CC3CCF8480000BFCF4879
S3150000C910407DE0B113F0020F19D10020DFF830C3DB
S3150000C920CCF8180000BF21210FE000BF2020DFF85F
S3150000C93024C3CCF8880000BF00BF00BF00BFCCF8FE
S3150000C940840000BF00BF00BF491E0029EDD10120B1
S3150000C950DFF8FCC2CCF8180000BFF0B29CE7BB4879
S3150000C960007D00F121010FE000BF2020DFF8E4C2C6
S3150000C970CCF8880000BF00BF00BF00BFCCF8840021
S3150000C98000BF00BF00BF491E0029EDD10120DFF81E
S3150000C990C0C2CCF8180000BFF0B27DE703B587B07F
S3150000C9A00020039001200190A9490198886100BFE9
S3150000C9B000BF2020A849086000BFA4484068019035
S3150000C9C00198009000BF00BF0098401E0090FBD168
S3150000C9D000BF00BF2020A149086000BF9B484068F7
S3150000C9E001900198009000BF00BF0098401E009083
S3150000C9F0FBD100BF079805900598019094490198CE
S3150000CA00886100BF00BF20219348016000BF8F48A6
S3150000CA10406801900198009000BF00BF0098401E3A
S3150000CA200090FBD100BF00BF20208C49086000BFEA
S3150000CA308648406801900198009000BF00BF0098AA
S3150000CA40401E0090FBD100BF05990398084403904F
S3150000CA50079840080590059801907D4901988861DE
S3150000CA6000BF00BF20207C49086000BF77484068AF
S3150000CA7001900198009000BF00BF0098401E0090F2
S3150000CA80FBD100BF00BF20207449086000BF6F487B
S3150000CA90406801900198009000BF00BF0098401EBA
S3150000CAA00090FBD100BF05990398084403900798AE
S3150000CAB0800805900598019065490198886100BF36
S3150000CAC000BF20206449086000BF604840680190AC
S3150000CAD00198009000BF00BF0098401E0090FBD157
S3150000CAE000BF00BF20205D49086000BF574840686E
S3150000CAF001900198009000BF00BF0098401E009072
S3150000CB00FBD100BF05990398084403900798C00815
S3150000CB100590059801904E490198886100BF00BFB5
S3150000CB2020204D49086000BF4848406801900198A0
S3150000CB30009000BF00BF0098401E0090FBD100BFD0
S3150000CB4000BF20204549086000BF4048406801906A
S3150000CB500198009000BF00BF0098401E0090FBD1D6
S3150000CB6000BF05990398084403900398019038493B
S3150000CB700198886100BF00BF20203749086000BFC8
S3150000CB803248406801900198009000BF00BF0098AD
S3150000CB90401E0090FBD100BF00BF20202F49086037
S3150000CBA000BF2A48406801900198009000BF00BF6E
S3150000CBB00098401E0090FBD100BF019024490198C7
S3150000CBC0886100BF00BF20202349086000BF1F48BE
S3150000CBD0406801900198009000BF00BF0098401E79
S3150000CBE00090FBD100BF00BF20201C49086000BF99
S3150000CBF01648406801900198009000BF00BF009859
S3150000CC00401E0090FBD100BF012001901049019801
S3150000CC10886100BF00BF20200F49086000BF0B4895
S3150000CC20406801900198009000BF00BF0098401E28
S3150000CC300090FBD100BF00BF20200849086000BF5C
S3150000CC400248406801900198009009E068F4FF1FCF
S3150000CC500010FE4300F00F4088F00F4084F00F40B4
S3150000CC6000BF00BF0098401E0090FBD100BF00BF70
S3150000CC700120FE49486400BFFD48007D029024E083
S3150000CC8000BF2020FB49086000BFF94840680190BA
S3150000CC900198009000BF00BF0098401E0090FBD195
S3150000CCA000BF00BF2020F449086000BFF04840687C
S3150000CCB001900198009000BF00BF0098401E0090B0
S3150000CCC0FBD100BF0298401E029002980028D7D1DF
S3150000CCD000BF2020E749086000BFE5484068019092
S3150000CCE00198009000BF00BF0098401E0090FBD145
S3150000CCF000BF00BFE1480068059000BF4FF020006C
S3150000CD00DA49C1F8840000BFD9484068019001980B
S3150000CD10009000BF00BF0098401E0090FBD100BFEE
S3150000CD200598069000BF2020D249086000BFD04871
S3150000CD30406801900198009000BF00BF0098401E17
S3150000CD400090FBD100BF00BFCC480068059000BF33
S3150000CD504FF02000C549C1F8840000BFC4484068B0
S3150000CD6001900198009000BF00BF0098401E0090FF
S3150000CD70FBD100BFDDE9051040EA4100069000BF87
S3150000CD802020BC49086000BFB9484068019001985E
S3150000CD90009000BF00BF0098401E0090FBD100BF6E
S3150000CDA000BFB6480068059000BF4FF02001AF48AD
S3150000CDB0C0F8841000BFAE4840680190019800900A
S3150000CDC000BF00BF0098401E0090FBD100BFDDE908
S3150000CDD0051040EA81000690069801287CD1079844
S3150000CDE010F0020F79D000200490039020200290CA
S3150000CDF036E000BF20209F49086000BF9C4840687D
S3150000CE0001900198009000BF00BF0098401E00905E
S3150000CE10FBD100BF00BF99480068059000BF4FF0E6
S3150000CE2020009249C1F8840000BF914840680190F3
S3150000CE300198009000BF00BF0098401E0090FBD1F3
S3150000CE4000BF05990398084403900498400804908D
S3150000CE50DDE9040140EAC17004900298401E029088
S3150000CE6002980028C5D100BF20208249086000BF73
S3150000CE707F48406801900198009000BF00BF00986D
S3150000CE80401E0090FBD100BF00BF7C4800680590A3
S3150000CE9000BF4FF020007549C1F8840000BF7448F8
S3150000CEA0406801900198009000BF00BF0098401EA6
S3150000CEB00090FBD100BF05990398484010F0010F80
S3150000CEC001D008200690089810B1089904980860C7
S3150000CED06748007D029026E00FE12DE000BF20208C
S3150000CEE06449086000BF624840680190019800905C
S3150000CEF000BF00BF0098401E0090FBD100BF00BFDE
S3150000CF0020205D49086000BF59484068019001989B
S3150000CF10009000BF00BF0098401E0090FBD100BFEC
S3150000CF200298401E029002980028D7D100BF012027
S3150000CF304E49886400BF95E04D48007D029024E08C
S3150000CF4000BF20204B49086000BF49484068019057
S3150000CF500198009000BF00BF0098401E0090FBD1D2
S3150000CF6000BF00BF20214448016000BF4048406820
S3150000CF7001900198009000BF00BF0098401E0090ED
S3150000CF80FBD100BF0298401E029002980028D7D11C
S3150000CF9000BF01213548816400BF089800680490ED
S3150000CFA0002003902020029031E00498019034493B
S3150000CFB00198886100BF00BF20202E49086000BF8D
S3150000CFC02B48406801900198009000BF00BF009870
S3150000CFD0401E0090FBD100BF00BF202026490860FC
S3150000CFE000BF2348406801900198009000BF00BF31
S3150000CFF00098401E0090FBD100BFDDE90301084404
S3150000D00003900498400804900298401E02900298EB
S3150000D0100028CAD10398019019490198886100BF78
S3150000D02000BF20201349086000BF114840680190E6
S3150000D0300198009000BF00BF0098401E0090FBD1F1
S3150000D04000BF00BF20210C48016000BF08484068AF
S3150000D05001900198009000BF00BF0098401E00900C
S3150000D060FBD100BF0248007A02900BE000F00F40AF
S3150000D07068F4FF1F88F00F4084F00F401C12FE4337
S3150000D0800010FE43029870B3002001909449019865
S3150000D090886100BF24E000BF20209249086000BFDD
S3150000D0A09148406801900198009000BF00BF009829
S3150000D0B0401E0090FBD100BF00BF20208B490860B6
S3150000D0C000BF8948406801900198009000BF00BFEA
S3150000D0D00098401E0090FBD100BF0298401E0290AF
S3150000D0E002980028D7D1012001907D4901988861D6
S3150000D0F000BF0698C0B209B000BD0698022802D04B
S3150000D1000698042873D17848407D70B3079810F0CC
S3150000D110020F2AD02120029024E000BF202171486E
S3150000D120016000BF7048406801900198009000BF00
S3150000D13000BF0098401E0090FBD100BF00BF20201A
S3150000D1406A49086000BF68484068019001980090ED
S3150000D15000BF00BF0098401E0090FBD100BF0298A0
S3150000D160401E029002980028D7D15F48007D0290A9
S3150000D17024E000BF20215B48016000BF5A48406898
S3150000D18001900198009000BF00BF0098401E0090DB
S3150000D190FBD100BF00BF20205449086000BF5248A1
S3150000D1A0406801900198009000BF00BF0098401EA3
S3150000D1B00090FBD100BF0298401E02900298002802
S3150000D1C0D7D100BF012049498439886400BF464849
S3150000D1D0407DA8B3079810F0020F31D100200190CE
S3150000D1E03F490198886100BF2120029025E030E088
S3150000D1F000BF20203B49086000BF3B4840680190C3
S3150000D2000198009000BF00BF0098401E0090FBD11F
S3150000D21000BF00BF20203549086000BF3248406883
S3150000D22001900198009000BF00BF0098401E00903A
S3150000D230FBD100BF0298401E029002980028D7D169
S3150000D2400120019026490198886100BF0698C0B266
S3150000D25051E72548007D2130029024E000BF2020C0
S3150000D2602049086000BF204840680190019800905E
S3150000D27000BF00BF0098401E0090FBD100BF00BF5A
S3150000D28020201A49086000BF17484068019001989D
S3150000D290009000BF00BF0098401E0090FBD100BF69
S3150000D2A00298401E029002980028D7D101200190D2
S3150000D2B00B490198886100BF0698C0B21BE730B5DC
S3150000D2C004460D460848407820B129462046FFF717
S3150000D2D0E4F830BD29462046FFF760FBF9E7000079
S3150000D2E00010FE4388F00F4068F4FF1F84F00F40E3
S3150000D2F0704770477047024600207047024600207C
S3150000D3007047704770477047F0B502460B680C6867
S3150000D3109C4201DD1C4600E00C68234618460DE0E1
S3150000D320F94C2478641EF94D2E682D686D1CF74F54
S3150000D33034403D60F64D2C5D02F8014B1C00A3F114
S3150000D3400103EDD1F0BDF0B502460B46196808465B
S3150000D35010E012F8016BEC4C2478641EED4D2F683A
S3150000D3602D686D1CDFF8ACC33C40CCF80050E84D8E
S3150000D3702E55491E0029ECD1F0BD0146E248007841
S3150000D380401EE44A1268E14B1B68D21A104008603E
S3150000D3900020704708B50020DF4908806846FBF783
S3150000D3A0EAFEBDF8000010F4004F05D0DA48008808
S3150000D3B040F00100D8490880BDF8000010F4005F75
S3150000D3C005D0D548008840F00200D3490880BDF852
S3150000D3D0000010F0100F05D0CF48008840F0040080
S3150000D3E0CD490880BDF8000010F4804F05D0CA482A
S3150000D3F0008840F00800C8490880BDF8000010F019
S3150000D400080F05D0C448008840F01000C2490880C3
S3150000D410BDF8000010F0040F05D0BF48008840F0AA
S3150000D4202000BD490880BDF8000010F0020F05D0AD
S3150000D430B948008840F04000B7490880B6480088DF
S3150000D44008BD10B5FBF702FDB44C23796279A179CA
S3150000D4502068FBF729FD0120B1490880FFF79AFFF4
S3150000D460AD4908800020AB490860A849086010BD96
S3150000D4700120704701207047014601207047014690
S3150000D4800120704701460120704710B5A548007875
S3150000D490A449497840EA0120A249897840EA014036
S3150000D4A0A049C97840EA01609C4908609D48007916
S3150000D4B008719C48407948719A4880798871FBF7D1
S3150000D4C0DFFCFBF7C3FC012095490880934C2379C8
S3150000D4D06279A1792068FBF7E7FC012010BD8F482F
S3150000D4E00078904908708D480088000A48708B487B
S3150000D4F00068000C887089480068000EC87087486C
S3150000D5000079087185484079487184488079887126
S3150000D5100120704701460120704710B50446204699
S3150000D520FBF792FD012010BD38B56846FBF7E1FD1B
S3150000D5300020FDF7F9F869467B48FBF72DFD044608
S3150000D540002C08DD7949097841F0800022467649A9
S3150000D550FBF754FB02E001207149088038BD10B585
S3150000D5600020FDF7E1F868480078401E694909681F
S3150000D570664A1268891A084063490978081A6C498C
S3150000D5800978884203D801206A49088010BD6A4993
S3150000D5906A480078FBF7A3FA694908606648FFF70E
S3150000D5A0D2FE00BFF2E710B5A12066490870202020
S3150000D5B0487000208870C870087148710220887110
S3150000D5C00020C87154480078087253480088000A41
S3150000D5D048725D49097841F080000A225949FBF7F3
S3150000D5E00DFB10BD38B56846FBF783FD0098002893
S3150000D5F012DD4B48008878B169465448FBF7CCFCED
S3150000D60004460020464908804849097841F08000D0
S3150000D61022464E49FBF7F2FA38BD70B504460D4670
S3150000D62003E00220DFF828C100DF3D48008800281B
S3150000D630F7D000203A4908803C49097841F080003B
S3150000D6402A462146FBF7DAFA70BD0EB56846FFF7A3
S3150000D65094FE009800280FDD0098202801DD202088
S3150000D66000E00098029002A93A48FFF74DFE0190AB
S3150000D67001A93848FBF713FD0EBD10B5FFF78AFE6A
S3150000D680044635480088A04203D033480480FFF79B
S3150000D6908AFF10BD10B52748008850B11B480068A6
S3150000D6A01C490968884204D1002022490880FFF7F6
S3150000D6B056FF10BD70B5054615F0080F0AD0FFF7E6
S3150000D6C069FE044625480088A04203D0234804800A
S3150000D6D0FFF769FF70BD10B50446FFF725FF10BDC3
S3150000D6E010B50446FFF73BFF10BD10B5044614F015
S3150000D6F0040F02D02046FFF7F3FF14F0080F02D004
S3150000D7002046FFF7E8FF10BDCC090100E4E0FF1F4B
S3150000D71022090020E0E0FF1FD0E0FF1FC8E0FF1F46
S3150000D720D2E0FF1F0CE0FF1F62080020C9090100BC
S3150000D730CB090100D4E0FF1FA2080020CA0901009E
S3150000D740DCE0FF1FA0F4FF1FC8090100E20800206B
S3150000D7509101010080F4FF1FD6E0FF1FD8E0FF1FF4
S3150000D7602048006858B100BF4FF6FF710846FBF726
S3150000D7700DFEFBF707FE0446FFF79CFFF4E719488A
S3150000D780006870B100BF4FF6FF710846FBF7FEFD5B
S3150000D790FBF7F8FD10F0080FF5D00020FFF79BFF10
S3150000D7A0F1E71048006870B100BF4FF6FF710846F8
S3150000D7B0FBF7ECFDFBF7E6FD10F0040FF5D00020BB
S3150000D7C0FFF78EFFF1E70748006858B100BF4FF634
S3150000D7D0FF710846FBF7DAFDFBF7D4FD0446FFF7B9
S3150000D7E084FFF4E7380A010010B50020F7490870F5
S3150000D7F0FBF7D1FDFBF7D8FDFAF7E2FF10BD10B538
S3150000D80004462046FBF731F810BDF1480078F1498F
S3150000D81008800020F0490870F04908704FF00110A8
S3150000D820EF4908600020EF490860EF49086070473B
S3150000D830EA48007808B1012070470020FCE710B5DF
S3150000D840EA490020FBF74BF910BD10B5E84880887F
S3150000D850E8490978884202DDE648047801E0E448B0
S3150000D860848814B90020E4490870E148224601681A
S3150000D8708020FBF7C3F90446DD4800682044DC49F4
S3150000D880086008468088001B888010BD10B5D848FF
S3150000D89001680020FBF723F90446D54800682044B8
S3150000D8A0D349086008468088001B888010BD10B5E3
S3150000D8B0002211468020FBF7A1F910BD10B5CF4913
S3150000D8C00020FBF70CF910BD10B5044614F0020F4A
S3150000D8D076D0FFF7B4FFC5490978C809FBF7B2F857
S3150000D8E0C248C088C2498880C0480078C0F3411049
S3150000D8F010B1012877D1D9E0BC4840780C2873D202
S3150000D900DFE800F0060DD127D1415F66677C95B848
S3150000D91002F0B8F800B9F9E0FFF797FFC4E000207D
S3150000D92002F010F900B9F1E0FFF7C1FFB448006852
S3150000D93040B1B448006858B1B24801680820FBF706
S3150000D9401BFD05E0B048006810B1AF48006880478D
S3150000D950AAE0012002F0F6F800B9D7E0FFF7A7FF2A
S3150000D960A748006840B1A748006858B1A5480168B3
S3150000D9700420FBF701FD05E0A348006810B1A248AA
S3150000D9800068804790E000BF9848007810F01F0FAD
S3150000D99006D19648807840F080008F49087001E0F3
S3150000D9A0002001E000BF012000B9AFE08A490978F4
S3150000D9B001F07F000121FAF7D6FFFFF778FF73E049
S3150000D9C0B7E001F06DFF00B9A0E0FFF73EFF6BE0A6
S3150000D9D09CE000BF8548007810F01F0F05D17F48F6
S3150000D9E08349086003E090E05DE0002001E000BFAD
S3150000D9F0012000B98AE0FFF728FF55E002F01AF986
S3150000DA0000B983E0FFF753FF7D48006840B17D48C9
S3150000DA10006858B17B4801680120FBF7ADFC05E0C2
S3150000DA207A48006810B17948006880473CE000BF3A
S3150000DA306E48007800F01F00012812D16748007870
S3150000DA4060B16A48007972490978884206DA6748FF
S3150000DA500079704908446649086001E0002004E046
S3150000DA6001E0002001E000BF012000B94EE0FFF711
S3150000DA70ECFE19E002F0D0F900B947E0FFF717FF16
S3150000DA805F48006840B15F48006858B15D4801686A
S3150000DA900220FBF771FC05E05F48006810B15E48A4
S3150000DAA00068804700E031E000BF41E04F48007861
S3150000DAB010F01F0004D0012807D0022823D119E056
S3150000DAC0FBF72CFC00B11FE020E000F0E5F900B107
S3150000DAD01AE000F07BFA00B116E0FBF717FC00B184
S3150000DAE012E000F0E7F800B10EE0FBF719FC00B118
S3150000DAF00AE00BE0FBF70CFC00B105E0FBF712FCBB
S3150000DB0000B101E002E001E012E000BF3748007812
S3150000DB10C00906D13548C08818B10020FAF7C1FF00
S3150000DB2002E08020FAF7BDFF00203149888000BF5F
S3150000DB3000BF14F0040F74D02C480078C0096ED1D1
S3150000DB402B48808888B3FFF7A1FE2948808860BBF0
S3150000DB5026480078C0F3411010B101282DD100E00D
S3150000DB602CE02248007810F01F0004D0012807D0CE
S3150000DB70022820D115E0FBF7D7FB00B11CE01DE021
S3150000DB8000F0EEF900B117E0FBF7C4FB00B113E0BB
S3150000DB9000F006F900B10FE0FBF7C8FB00B10BE09F
S3150000DBA00CE0FBF7B9FB08B106E03AE0FBF7C0FB77
S3150000DBB000B101E002E001E007E000BF8020FAF7D3
S3150000DBC070FF00200A49888000BF2AE0F9E0FF1FA5
S3150000DBD0A4090100E8E0FF1FEAE0FF1FEBE0FF1FDA
S3150000DBE0ECE0FF1FF0E0FF1FF4E0FF1F04E1FF1F62
S3150000DBF0FCE0FF1FA9090100FAE0FF1F0CE0FF1F70
S3150000DC00380A010010E1FF1F340A01002C0A010046
S3150000DC10F8E0FF1F08E0FF1F300A0100FFE7FFF7EB
S3150000DC204DFE14F0080F1ED01D4800780121B1EBFF
S3150000DC30D01F08D11B48808810B91B48007890B1C6
S3150000DC40FFF703FE0FE01948007810F0800F0AD0A6
S3150000DC501648007800F07F00144908700021134828
S3150000DC600078FAF780FE14F0400F02D00020FAF791
S3150000DC7023FF14F0800F02D08020FAF71DFF10BD9D
S3150000DC800B48006858B100BF4FF6FF710846FBF716
S3150000DC907DFBFBF777FB0446FFF716FEF4E7000073
S3150000DCA004E1FF1FFCE0FF1FFAE0FF1FEAE0FF1F91
S3150000DCB0380A010010B5534800795349097888425B
S3150000DCC005D05048007951490978884266D14D48B7
S3150000DCD04078042833D007DC78B1012812D0022816
S3150000DCE01BD0032859D11DE0202832D0212835D059
S3150000DCF022283ED0232850D145E0454845490860B2
S3150000DD00012010BDFFF7B6FB30B14148414908601C
S3150000DD10FFF79BFD0120F4E73FE03D483D490860E1
S3150000DD200120EEE737494888FFF7A9FB30B13848AC
S3150000DD3038490860FFF789FD0120E2E72DE0314907
S3150000DD404888FFF79FFB18B1FFF7B1FD0120D8E720
S3150000DD5023E02F482F4908600120D2E7FFF7BFFBD9
S3150000DD6030B12B482B490860FFF76FFD0120C8E74B
S3150000DD7013E024494888FFF7CDFB18B1FFF797FD5C
S3150000DD800120BEE709E01F494888FFF7C6FB18B126
S3150000DD90FFF78DFD0120B4E700BF00BF0020B0E70C
S3150000DDA010B51848007918490978884205D01548F1
S3150000DDB0007916490978884222D11248407820B164
S3150000DDC002280AD020281AD111E0FFF751FB18B11A
S3150000DDD0FFF76DFD012010BD11E00A494888FFF7E5
S3150000DDE04BFB18B1FFF763FD0120F4E707E0FFF7EF
S3150000DDF04CFB18B1FFF75BFD0120ECE700BF00BF4D
S3150000DE000020E8E704E1FF1FC6090100C709010079
S3150000DE100CE0FF1FFCE0FF1F02465C48C07821288B
S3150000DE2004D0222822D0232831D12EE05748007969
S3150000DE30574B1B78984201D0002070475548007810
S3150000DE4028B955480078012801D10020F5E7524845
S3150000DE50007810B95148106001E051481060106810
S3150000DE601230504B18600920086012E047480079CC
S3150000DE70474B1B78984201D00020DEE74A48494BC1
S3150000DE8018604A480088086003E00020D5E70020B3
S3150000DE90D3E700BF0120D0E710B53C4800793C49E4
S3150000DEA0097888425AD1394840780C2855D2DFE89B
S3150000DEB000F054062E4154545454541D394C00F06D
S3150000DEC0C8F890B13148C078012803D1384835499F
S3150000DED0086006E02D48C078032802D1354831494C
S3150000DEE00860FFF7B2FC012010BD36E02748C07875
S3150000DEF0022803D130482B49086006E02348C07841
S3150000DF00032802D12B48274908600120ECE700F0DE
S3150000DF10D8F830B1294823490860FFF796FC01205C
S3150000DF20E2E71AE000F0D5F818B1FFF7C0FC0120CF
S3150000DF30DAE712E000F0E5F830B120481949086048
S3150000DF40FFF783FC0120CFE707E000F0E1F818B106
S3150000DF50FFF7ADFC0120C7E700BF00BF0020C3E705
S3150000DF6010B50A4800790A49097888420CD1074851
S3150000DF704078092807D100F087F818B1FFF797FC19
S3150000DF80012010BD00BF00BF0020FAE704E1FF1F1B
S3150000DF90AA090100A5090100F9E0FF1FCE0A010048
S3150000DFA0490B0100FCE0FF1F840A0100A60A0100DC
S3150000DFB0A10700201AE0FF1FE20700200CE0FF1F68
S3150000DFC010B50446204600F08BFB10BD10B517486F
S3150000DFD0007917490978884226D114484078FE28E6
S3150000DFE00FD0FF281FD11148408848B90F48C08874
S3150000DFF030B900F09FFB18B1FFF759FC012010BDA6
S3150000E00011E00A48408868B90848C088012809D143
S3150000E01000F099FB30B1074807490860FFF715FC87
S3150000E0200120ECE700BF00BF0020E8E704E1FF1F86
S3150000E030BE0901000CE0FF1FFCE0FF1F704710B592
S3150000E0400446002010BD10B5029C10BD002070478C
S3150000E050704710B50024FE48C078012804D0022875
S3150000E06004D0032806D103E0FA4C03E0002010BDDB
S3150000E070F94C00BF00BFF64A9178D07800232246BB
S3150000E080FBF7EEF90120F2E738B50024F048C07836
S3150000E090012804D0022804D0032806D103E000207A
S3150000E0A038BDEE4C01E0EC4C00BF00BF0020E84A52
S3150000E0B00090D3889178D0782246FBF717FA012092
S3150000E0C0EEE7E3488078E649085CE64908700120F7
S3150000E0D07047DF48807830B1DD48C2788078401ECE
S3150000E0E0DF4B1A540BE0002105E0D948C078DC4A22
S3150000E0F05054481CC1B2DC4800788142F5DB01204F
S3150000E100704710B5FFF7A2FFD6490870012010BD71
S3150000E11010B5CF498878FFF79BFF012010BD70B579
S3150000E1200646D2480088D2490988884226DBD1486B
S3150000E130006818BB0020D0490860CC490880C54853
S3150000E140401E01780123421C1846FBF789F9C8498D
S3150000E15008800846008888B1BE48401EC649086047
S3150000E160C1480078012804DC08460068401C0860A5
S3150000E17004E0BF480088401CBD490880BC480088B0
S3150000E18000285FD1BD48006818B10020BB4908606F
S3150000E19058E0BB480068002854D0B34800780128EE
S3150000E1A01BDCB748006800284CD00020A949491E4E
S3150000E1B00870AE4908800223A64A00210120FBF719
S3150000E1C04FF9AB4908800846008810B1A148AA4912
S3150000E1D008600020AA49086034E09E48401E047882
S3150000E1E000BF202C00DB00240120A040A4490968C0
S3150000E1F0084223D0601C9749491E087000209B499D
S3150000E2000880601CC1B20223924A0120FBF728F95C
S3150000E210974908800846008840B18E48401E9649B6
S3150000E220086093480088401C914908800120A0405E
S3150000E2309349096881439248016002E0601CC4B2B8
S3150000E240CFE700BF8A48008810B98A480068A0B3A3
S3150000E2508748008885490988401A85B289488A49CD
S3150000E260097830F81100A84204DA86488649097808
S3150000E27030F811508549097841F080002A467E49D8
S3150000E2800968FAF7BBFC7C48006828447A490860AC
S3150000E29076480088284475490880084600887C49E5
S3150000E2A0098888420ADA77487749097830F81100F0
S3150000E2B0A84203D101206F49086002E000206D49A1
S3150000E2C0086070BD38B505467248008830B96348A5
S3150000E2D0401E7149086000206E4908806E4801683A
S3150000E2E06E480078FAF7FBFB84B26B48006820445E
S3150000E2F0694908606748008820446649088064B117
S3150000E3000846008866490988884206DA5D485E49FB
S3150000E310097830F81100A0421DDD62480078012816
S3150000E3200ADC012000905B4803884C4A521E0021FB
S3150000E3300220FBF7DBF80BE001200090554800882F
S3150000E340431E4648401E0178421C0220FBF7CEF8C9
S3150000E35000205049088038BD0020534908704749BD
S3150000E36008604749086044490860414908803F49B8
S3150000E37008804049086048490860464908804B497A
S3150000E38008604B490880704710B5044614F0080F22
S3150000E39002D02046FFF7C3FE14F0040F02D0204639
S3150000E3A0FFF790FF10BD2DE9F041424800780028A4
S3150000E3B04CD00026404801780078401C3E4A107038
S3150000E3C03148007800EB400204209040401E814214
S3150000E3D003DB0020384908700126002537480088ED
S3150000E3E0FF2804DA35480088401C34490880344840
S3150000E3F02549097830F8110030490988884200D14A
S3150000E40001250024A1E04FF000089EB12D48005DD3
S3150000E410FF2804DA2B48005D401C2A4908552A4883
S3150000E420005D38B12748005D2749095D884201DB58
S3150000E4304FF001082448005D1349097801EB4102B9
S3150000E4400221914088401E490F4A3FE08FE00000BC
S3150000E45004E1FF1FA10700201AE0FF1FE2070020CA
S3150000E46018E0FF1F0CE0FF1FB60901006E00002038
S3150000E4706C00002070000020680000206000002072
S3150000E48064000020B2090100F9E0FF1FAB0901009A
S3150000E490B80901007800002074000020AC090100D2
S3150000E4A0BA090100B70901005D0000207C000020C8
S3150000E4B080000020EBE0FF1F5C00002014E0FF1F3F
S3150000E4C0AE09010016E0FF1F17E0FF1F127831F8B2
S3150000E4D01210884204DA6648005D08B1012000E0A7
S3150000E4E0002007463DB137B10120A04061490968C7
S3150000E4F00843604908605E48005D5F49095D8842DF
S3150000E50013D05E48005D5C49095D884209DB012045
S3150000E510A0405849096808435649086000205849F0
S3150000E52008705548005D52490855B8F1000F0AD0E9
S3150000E53037B90120A0404F49096808434D49086092
S3150000E54000204E490855601CC4B24E4800788442EB
S3150000E550FFF659AF15B100204B49088045480068C1
S3150000E56028B14A48008810B90020FFF7D8FDBDE859
S3150000E570F0814748006870B100BF4FF6FF7108464A
S3150000E580FAF704FFFAF7FEFE10F0080FF5D00020A8
S3150000E590FFF7C5FDF1E73E48006870B100BF4FF6D2
S3150000E5A0FF710846FAF7F2FEFAF7ECFE10F0040FD8
S3150000E5B0F5D00020FFF786FEF1E73548006858B130
S3150000E5C000BF4FF6FF710846FAF7E0FEFAF7DAFEEB
S3150000E5D00446FFF7D9FEF4E770B504460E46154625
S3150000E5E02C480088854201DD002070BD2A4800784D
S3150000E5F000283AD00120294908600CE02648007816
S3150000E60048B9002025490860254908602549088041
S3150000E6101E490880E9E71D4800880028EED12248F7
S3150000E62004702A463146401C01F036F81E481C4943
S3150000E630086000201B49088014490D8011480078A5
S3150000E640012805DC16480068401C1549086004E0EE
S3150000E6500E480088401C0D4908800020FFF75FFD2A
S3150000E6600020064908550120BFE70020BDE700004D
S3150000E67017E0FF1F6400002018E0FF1F16E0FF1FD1
S3150000E6805C000020B609010014E0FF1F6C000020AA
S3150000E690380A0100B8090100EBE0FF1F6000002006
S3150000E6A0680000206E000020A00700207047704719
S3150000E6B07047704710B504462046FAF7F2F914F091
S3150000E6C0800F05D004F00F014FF48030884001E040
S3150000E6D00120A040FE4909680843FD49086010BDB5
S3150000E6E070B50646FB48007900F08F0414F0800FE1
S3150000E6F005D004F00F014FF48030884001E001207E
S3150000E700A0400546F448007840F08000A04210D1B1
S3150000E710EF48006828420CD0F0480068F04988426B
S3150000E72007D1ED49097841F080000D22EB49FAF74F
S3150000E73065FA70BD0020EB490860E8490860EA49BF
S3150000E7400870012070470020E849087001207047D2
S3150000E75010B5E348E1490860DF49097841F08000D7
S3150000E7600D22DE49FAF74AFA0520DF49087010BD86
S3150000E77010B5DF480068DF490860DD480068C8B9A1
S3150000E780DD48806878B1DC48007B10F0800F06D049
S3150000E790D149097841F08000FFF78CFF03E0D748A4
S3150000E7A00078FFF787FF0120CC490873FFF7D0FFF9
S3150000E7B0002010BD0120FCE770B5D1480068D149A2
S3150000E7C0096888420CD30024C349097841F08000C7
S3150000E7D0FFF770FF0020C1490873FFF7B9FF10E08B
S3150000E7E0C948CA49097830F81100C94909688842F8
S3150000E7F005D2C548C549097830F8114001E0C4483A
S3150000E8000468FFF7B5FF00B90024C2480068B8B92C
S3150000E810B4B1C1480068401EBD4909680844BE49F4
S3150000E8200968B0FBF1F5BD480068854201D9BB48CF
S3150000E83005682A46BA480168B1480068FBF799FAA4
S3150000E840ACB1B74A1268B34B1B68D118A24A12780A
S3150000E85042F080002246FAF7D1F9AE48006820441B
S3150000E860AC490860AA480068001BA9490860AB4883
S3150000E8700068A94909684843A6490968884209D138
S3150000E8800020A44908609E480068A4490968084415
S3150000E8909B49086091488068001B9049886004B9CC
S3150000E8A070BD9B48006810B903208F4908708E48D8
S3150000E8B00078022802D000208849087300BFEFE7DD
S3150000E8C010B58F4800688F49096888420BD300202D
S3150000E8D09449086089480078FFF7ECFE00207F49DC
S3150000E8E00873FFF735FFFFF743FF10B900208D4986
S3150000E8F00860002408E08C48005D864909682144C8
S3150000E900874A12685054641C864800688442F2D3D1
S3150000E910804800688349096808447E4908607C4845
S3150000E920006880490968401A794908607D4800688E
S3150000E930002840D00846006810BB76480068F8B149
S3150000E94075480068401E7349096808447249096899
S3150000E950B0FBF1F471480068844201D96F4804683D
S3150000E96022466F48016866480068FBF7A9FA00204E
S3150000E97068490860624800682044614908601AE0F6
S3150000E98066480068644909684843624909688842DC
S3150000E99011D1624802686248016859480068FBF76D
S3150000E9A08FFA00205B490860554800685B49096892
S3150000E9B0084453490860494880685A490968401A1A
S3150000E9C0464988605748006800B910BD504800683D
S3150000E9D018B145480078052804D100203F4908733E
S3150000E9E0FFF7B6FE00BFF0E710B545480068454999
S3150000E9F0096888420BD300204A4908603F480078DE
S3150000EA00FFF758FE002035490873FFF7A1FEFFF710
S3150000EA10AFFE10B90020434908604248006800284C
S3150000EA2032D03C480068C8B93E480068B0B13A48A0
S3150000EA300068401E36490968084437490968B0FB32
S3150000EA40F1F436480068844201D934480468224605
S3150000EA50334801682A480068FBF78BF900240EE06A
S3150000EA602C48006820442E490968085C2E49095D37
S3150000EA70884203D000202D49086004E0641C294820
S3150000EA8000688442ECD300BF224800682549096823
S3150000EA900844204908601E48006822490968401A4F
S3150000EAA01B4908601D4800681B4909684843194905
S3150000EAB00968884209D10020164908601048006894
S3150000EAC01649096808440E490860044880682FE022
S3150000EAD0F0E0FF1F04E1FF1FBF090100071400203B
S3150000EAE055534253F4E0FF1FB40000200CE0FF1F13
S3150000EAF0840000208C000020E8130020C0090100DB
S3150000EB00A80000209C000020C2090100F9E0FF1FB8
S3150000EB10B0000020AC0000209400002098000020E7
S3150000EB20A0000020B800002022080020A400002039
S3150000EB30FE490968401AFE498860FC48006800B929
S3150000EB4010BDFC48006818B1FB480078052809D1BB
S3150000EB50FA48006808B9012000E00020F44908736B
S3150000EB60FFF7F6FD00BFEBE710B5F548407C010660
S3150000EB70F348807C41EA0041F148C07C41EA00202C
S3150000EB80EF49097D40EA0104EE4804600020EE49A1
S3150000EB900860EB48C07B2F280BD004DC28280ED059
S3150000EBA02A2828D104E0A82815D0AA2823D10CE0C9
S3150000EBB000BFFFF7DDFD08B9002010BD00BFE0482B
S3150000EBC0C17D807D41EA002415E0FFF7D1FD08B93B
S3150000EBD00020F2E700BFDA48407D0106D848807D74
S3150000EBE041EA0041D648C07D41EA0020D449097E69
S3150000EBF040EA010400BF00BFD44800686043CD4925
S3150000EC000860CF48806830B90120C9490873FFF70A
S3150000EC109FFD0020D1E7CA488068C6490968884236
S3150000EC2016D0C748007B10F0800F06D0C849097877
S3150000EC3041F08000FFF73EFD03E0C6480078FFF78D
S3150000EC4039FD0120BA490873FFF782FD0020B4E7B9
S3150000EC500120B2E710B5BA48806830B90220B4493D
S3150000EC600873FFF775FD002010BDB548007B10F056
S3150000EC70800F0AD1B7480078FFF71CFD0220AC4987
S3150000EC800873FFF765FD0020EEE70120ECE710B5FD
S3150000EC90AB488068A5490968884207D8A8488068B3
S3150000ECA0A24908600320A449087002E00420A24992
S3150000ECB00870A749097841F080009C490A68A6496E
S3150000ECC0F9F79CFF9A48806898490968401A98495C
S3150000ECD088600020087310BD10B599488068A8B1F7
S3150000ECE09748007B10F0800F06D09949097841F0CB
S3150000ECF08000FFF7DFFC03E096480078FFF7DAFCB8
S3150000ED0001208B490873FFF723FD10BDFFF730FD87
S3150000ED1000B9FAE7002086490873FFF719FD00BF1E
S3150000ED20F3E710B5FFF796FF00B910BD70208A49CA
S3150000ED300870002048708948006889490968484079
S3150000ED408749096808420BD0062083498870282025
S3150000ED5008730020487382480068804908601AE0FA
S3150000ED607F48006838B902207B4988703A200873CA
S3150000ED70002048730FE06E48007B28B900207649D2
S3150000ED8088700873487306E0052073498870202050
S3150000ED9008730020487300206F49C87008714871D5
S3150000EDA088710A20C8710020087248728872C87279
S3150000EDB08873C8730874487412205C490860FFF7AA
S3150000EDC066FF00BFB1E770B5FFF744FF00B970BD3D
S3150000EDD0FFF7CEFC00B9FAE700205F4908708020F3
S3150000EDE0487002208870C870202008710020487181
S3150000EDF08871C8715B48056808240BE0287820B143
S3150000EE0015F8010B5449085502E0202052490855CF
S3150000EE10601CC4B2242CF1DB242044490860FFF7AF
S3150000EE2036FF00BFD3E710B54548807C78B9444823
S3150000EE30C07C00F001004A49086008460068FFF7F8
S3150000EE4038FC00203A490873FFF782FC10BD012008
S3150000EE5037490873FFF77CFC00BFF7E710B5384861
S3150000EE60C07C10F0010F03D001203149087302E085
S3150000EE7000202F490873FFF76BFC10BD10B5FFF794
S3150000EE80E9FE00B910BDFFF773FC00B9FAE70320ED
S3150000EE90314908700020487033480078C007000EDA
S3150000EEA088700020C87004202049086020488068C7
S3150000EEB00968884207D91D480068214988601B48AF
S3150000EEC000681B498860FFF7E2FE00BFDAE710B56D
S3150000EED0FFF7C0FE00B910BDFFF74AFC00B9FAE71C
S3150000EEE000201D49087006204870002088701E48C2
S3150000EEF00078C007000EC87000200871487188713C
S3150000EF00C87108200949086009488068096888426C
S3150000EF1007D9064800680A49886004480068044919
S3150000EF208860FFF7B4FE00BFD5E70000B8000020F8
S3150000EF3007140020B0000020B4000020A400002028
S3150000EF40E8130020A8000020AC0000209400002058
S3150000EF50BF090100C0090100220800208C00002022
S3150000EF608400002004E0FF1F8800002010B5FFF792
S3150000EF7071FE00B910BDFFF7FBFB00B9FAE7FB48CD
S3150000EF800068401E000EFA490870F8480068401EE6
S3150000EF90000C4870F5480088401E000A8870F34847
S3150000EFA00078401EC870F3480068000E0871F148EA
S3150000EFB00068000C4871EF480088000A8871ED4827
S3150000EFC00078C8710820EC490860FFF760FE00BFB2
S3150000EFD0D0E710B5FFF73EFE00B910BDFFF7C8FB3E
S3150000EFE000B9FAE70020E2490870487088700820E6
S3150000EFF0C870DE480068000E0871DC480068000C26
S3150000F0004871DA480088000A8871D8480078C871C3
S3150000F01002200872D7480068000C4872D54800885C
S3150000F020000A8872D3480078C8720C20D24908605A
S3150000F030D24880680968884207D9CF480068D04915
S3150000F0408860CD480068CD498860FFF720FE00BF84
S3150000F050C3E710B50020C9490873FFF779FB10BD57
S3150000F06010B5002404E0C248005DC5490855641C7B
S3150000F070C14800688442F6D3BF4800681F2879D18A
S3150000F080BF480068BF498842F9D1BD484068BB49BE
S3150000F0904860BB4880688860B948407B002807DC28
S3150000F0A0B748807B012803DBB548807B102806DD46
S3150000F0B000BF0120B1490873FFF74AFBCDE0B04815
S3150000F0C0C07B252844D013DC152836D007DC20B3B6
S3150000F0D0032825D0042826D012286FD124E01A2828
S3150000F0E02CD01B2823D01E2824D02328F5D12CE091
S3150000F0F0552826D008DC28282DD02A2845D02F28A8
S3150000F1005DD03528E9D180E05A281BD091287DD0E2
S3150000F110A82821D0AA287CD138E0FFF7DDFD79E0C8
S3150000F120FFF7FFFD76E0C4E7FFF74DFE72E0FFF75D
S3150000F1307AFE6FE0FFF792FE6CE0BAE7FFF79EFEFD
S3150000F14068E0B6E7FFF7C3FE64E0FFF742FF61E061
S3150000F150FFF70CFF5EE000BFFFF706FDA0B1884891
S3150000F160007B10F0800F06D0022087490870FFF759
S3150000F17023FB09E04FE085480078FFF79BFA022061
S3150000F1807E490873FFF7E4FA44E000BFFFF7ECFCA2
S3150000F19098B17B48007B10F0800F03D101207A499B
S3150000F1A008700AE07A49097841F08000FFF782FA90
S3150000F1B0022072490873FFF7CBFA2BE029E070486A
S3150000F1C0007C10F0020F05D100206C490873FFF790
S3150000F1D0BFFA1FE0FFF7C8FCB0B16948007B10F02A
S3150000F1E0800F06D10120684908706A4908600BE063
S3150000F1F00CE06749097841F08000FFF75BFA0220CE
S3150000F2005E490873FFF7A4FA04E000BFFFF721FF89
S3150000F21000E04EE721E05E49097841F08000FFF703
S3150000F22049FA5B48007800F00F014FF480308840BF
S3150000F2305949096808435849086054480078FFF757
S3150000F24039FA524801780120884053490968084331
S3150000F2505149086006204C49087010BD10B54A484F
S3150000F2600078022806D0032811D0042812D00528D9
S3150000F2701DD118E04248C07B282802D0A82804D116
S3150000F28000E000BFFFF798FA00BF00BF0FE0FFF7EE
S3150000F2905FFA0CE03E49097841F08000FFF70AFA70
S3150000F2A0FFF756FA03E000203749087000BF00BF99
S3150000F2B010BD10B53448007820B1012805D00528C6
S3150000F2C016D114E0FFF7CCFE1CE02D48C07B2A289F
S3150000F2D004D02F2806D0AA2807D100E000BFFFF7E8
S3150000F2E0EFFA02E0FFF780FB00BF00BF0AE009E08B
S3150000F2F026480078FFF7DEF9022020490873FFF759
S3150000F30027FA00BF00BF10BD10B50446FFF7A6FFE1
S3150000F31010BD10B5044616491C480078F9F7DFFB06
S3150000F32015490860FFF7C5FF10BD10B5044614F077
S3150000F330040F02D00020FFF7ECFF14F0080F02D0F4
S3150000F3400020FFF7E1FF10BD1448006840B300BF7E
S3150000F3504FF6FF710846FAF719F8FAF713F810F0A6
S3150000F360080FF5D00020FFF7CFFFF1E79C00002043
S3150000F3702208002094000020B80000200714002076
S3150000F380E813002055534243B4000020C009010091
S3150000F390BF090100A4000020F4E0FF1F380A0100A5
S3150000F3A0FFE71048006870B100BF4FF6FF710846CE
S3150000F3B0F9F7ECFFF9F7E6FF10F0040FF5D000209F
S3150000F3C0FFF7A7FFF1E70748006858B100BF4FF6FF
S3150000F3D0FF710846F9F7DAFFF9F7D4FF0446FFF79D
S3150000F3E0A4FFF4E7380A010070B504460D469C48B0
S3150000F3F000680422294603692046984770BD70B507
S3150000F40004460D4616469648006832462946436924
S3150000F4102046984770BD2DE9FE4380460D460020E4
S3150000F420009002A92846FFF7DFFF10B90020BDE8CB
S3150000F430FE8301A9281DFFF7D7FF08B90020F6E7CC
S3150000F440FAF795FF0446204600F04AF9061F02988F
S3150000F45008B90120EBE7701C0199814201D0012017
S3150000F460E5E7241D00270CE0029A511C10460122F4
S3150000F47002912146FFF7C3FF08B90020D7E7641CB5
S3150000F4807F1CB742F0D3012269460298FFF7B7FF07
S3150000F49008B90020CBE70020C8F800000120C6E725
S3150000F4A070B504460D460020FBF731F9002070BD0B
S3150000F4B038B505460C4669462046FFF795FF08B95C
S3150000F4C0002038BD0120FCE770B504460D46FBF769
S3150000F4D044F900202060012070BD70B504460D4639
S3150000F4E0FBF742F900202060012070BD10B55D4891
S3150000F4F004684FF0FF305B490860B4F5817F18D08F
S3150000F50006DC182C30D0A4F58070013835D107E020
S3150000F510B4F5827F16D0A4F5807005382DD11AE097
S3150000F520514801684F48FFF776FF08B9002010BD23
S3150000F53024E04D4801684B48FFF7B2FF08B90020A8
S3150000F540F5E71BE0484801684648FFF7BDFF08B9E4
S3150000F5500020ECE712E0444801684248FFF7BDFF8F
S3150000F56008B90020E3E709E03F4801683D48FFF796
S3150000F5709FFF08B90020DAE700E000BF00BF0120C6
S3150000F580D5E728E000224FF6FF710120DFF8DCC046
S3150000F59000DF00BF3248006833498268314890472F
S3150000F5A048B1FFF7A3FF50B12D480068C1682D4848
S3150000F5B00068884703E00220DFF8B4C000DF0022BD
S3150000F5C011460220DFF8A4C000DF0128E2D0294856
S3150000F5D0DFF8A4C000DFD5E7002028490860002135
S3150000F5E02448DFF89CC000DF00231A460221254884
S3150000F5F0DFF894C000DF25490860704710B51F4842
S3150000F600006800B110BD2148006800B9FAE7144847
S3150000F61000684168052088471C4801680120DFF81A
S3150000F62070C000DF01201549086000BFEAE71348F3
S3150000F630006800B970471548006800B9FAE7134832
S3150000F64001680220DFF848C000DF4FF6FF71094865
S3150000F650DFF840C000DF00200849086000BFE9E786
S3150000F6604C000020CC000020D000002051020100F8
S3150000F67091010100C00000205D060100C8000020C5
S3150000F6801D06010083F50000D9080100BC0000201A
S3150000F690F10101009506010040EA01039B0703D032
S3150000F6A009E008C9121F08C0042AFAD203E011F8BB
S3150000F6B0013B00F8013B521EF9D27047D2B201E07D
S3150000F6C000F8012B491EFBD270470022F6E710B561
S3150000F6D013460A4604461946FFF7F0FF204610BDBA
S3150000F6E00146002000E0401C0A5C002AFBD170475E
S3150000F6F030B480EA010202F0004530F0004221F009
S3150000F700004015D0A0B1C0F3C753C2F3C754C2F32B
S3150000F7101601C0F31600E41A41F4000140F4000299
S3150000F7207D34914201D3641C00E04900002C02DACA
S3150000F73030BC002070474FF400000023914201D3F3
S3150000F740891A034340084FEA4101F7D151B191426A
S3150000F75002D14FF0004105E002D24FF0010101E075
S3150000F7606FF0010103EBC450284430BC00F01EB812
S3150000F77096230022114600F022B800F0004220F045
S3150000F7800040C10DC0F3160040F400007F2901DAE5
S3150000F79000207047962903DCC1F19601C84001E0BC
S3150000F7A096398840002AF4D0404270470029A8BF05
S3150000F7B07047401C490008BF20F00100704710B494
S3150000F7C0B0FA80FC00FA0CF050EA010404BF10BC49
S3150000F7D0704749B1CCF1200421FA04F411FA0CF176
S3150000F7E018BF012121430843A3EB0C01CB1D0106E1
S3150000F7F0000A002BBEBF002010BC704700EBC350B0
S3150000F80010440029A4BF10BC7047401C490008BF23
S3150000F81020F0010010BC7047064C074D06E0E0687A
S3150000F82040F0010394E8070098471034AC42F6D341
S3150000F830F8F7EAFD8C170100CC17010070B501EB53
S3150000F840020410F8015B15F0070301D110F8013B23
S3150000F8502A1106D110F8012B03E010F8016B01F80C
S3150000F860016B5B1EF9D12B0705D40023521E0FD462
S3150000F87001F8013BFAE710F8013B02F10202A1EBA5
S3150000F880030303E013F8015B01F8015B521EF9D58F
S3150000F890A142D6D3002070BD01000000A58700005C
S3150000F8A01CB56A48007810F01F0002D0012877D1F5
S3150000F8B0ACE06648C078082873D2DFE800F0A304FD
S3150000F8C0207AA3A30A4C624862490860122000907D
S3150000F8D09AE06148007828B960480078012801D18B
S3150000F8E000201CBD5D48007818B95D48594908607C
S3150000F8F002E05C48574908600A20009084E05648B8
S3150000F900007828B955480078012801D10020E8E799
S3150000F9105248007810B95448019001E053480190CC
S3150000F920002408E00198007820B1019840880199E8
S3150000F93008440190641C45488078A042F2D10198A1
S3150000F940007808B90020CCE7424901980860019880
S3150000F9504088009058E04048007828B93F48007831
S3150000F960012801D10020BCE73C48007810B9404886
S3150000F970019001E03F480190002408E001980078DA
S3150000F98020B101984088019908440190641C2F48D1
S3150000F9908078A042F2D10198007818B90020A0E73B
S3150000F9A03CE02FE02B4901980860019840880090C0
S3150000F9B02AE03148019025488078032807D1FAF7D4
S3150000F9C0E2FC24490860FAF7D4FC00901CE000240D
S3150000F9D008E00198007820B1019800780199084460
S3150000F9E00190641C19488078A042F2D101980078F1
S3150000F9F008B9002075E71749019808600198007852
S3150000FA00009001E000206CE700BF09E0694601A80C
S3150000FA10FEF702FA08B9002063E701E0002060E77C
S3150000FA2000BF0C488088009988420CD90949009883
S3150000FA3088800846808811490978491E084202D103
S3150000FA4001200F49087001204BE7000004E1FF1F69
S3150000FA50A80A0100FCE0FF1FA5090100F9E0FF1F4D
S3150000FA60BA0A0100C40A0100CE0A0100490B0100CE
S3150000FA704A0B01004B0B01004C0B0100A9090100C8
S3150000FA80FAE0FF1F2748007810F01F0004D0012875
S3150000FA9006D0022841D116E02348244B18603EE0E8
S3150000FAA02348007860B11F480079224B1B789842A2
S3150000FAB006DA0020204B188018461C4B186001E01F
S3150000FAC0002070472BE01748007900F08F0111F0F5
S3150000FAD0800F05D001F00F034FF48030984001E00D
S3150000FAE00120884002461248007810B911F00F0F25
S3150000FAF010D11248006810420CD01148006810421C
S3150000FB0001D0012000E000200B4B18801846074B5F
S3150000FB10186001E00020D4E701E00020D1E700BF33
S3150000FB200120CEE704E1FF1FE8E0FF1FFCE0FF1F16
S3150000FB30EBE0FF1FF8E0FF1F0CE0FF1FECE0FF1FEC
S3150000FB40F0E0FF1F70B506463448007810F01F003D
S3150000FB5004D001281DD002285BD11CE02F48408824
S3150000FB60012813D146B1F8F7FDFE2D48008840F074
S3150000FB7002002B4908800BE00020F8F7F3FE284826
S3150000FB80008820F002002649088001E0002070BDB0
S3150000FB9041E00020FBE72148007900F08F0414F0D3
S3150000FBA0800F05D004F00F014FF48030884001E04B
S3150000FBB00120A04005461B48007838B314F00F0F0B
S3150000FBC024D019480068284220D014484088D8B963
S3150000FBD046B12046F8F765FF1448006828431349E4
S3150000FBE0086015E012480068284201D00120CEE7DF
S3150000FBF02046F8F761FF2046FEF7E2F90B48006859
S3150000FC00A8430A49086003E00020C0E70020BEE7D9
S3150000FC1001E00020BBE700BF0120B8E704E1FF1FB9
S3150000FC20E8E0FF1FEBE0FF1FECE0FF1FF0E0FF1F27
S3150000FC30F4E0FF1F2DE9F04100266A48007810F035
S3150000FC401F0F6FD16748807800286CD0664800780F
S3150000FC5030B966480078012802D10020BDE8F0815D
S3150000FC606248007808B9624D00E0624D7FE068782E
S3150000FC70022804D0042853D0052874D154E06879AA
S3150000FC8058498978884247D1564880785A49087039
S3150000FC9028795A490870002403E00020584908557D
S3150000FCA0641C584800888442F7D3012414E00120DC
S3150000FCB0A04055490968084202D02046F8F7DAFE06
S3150000FCC04FF48030A04050490968084203D044F000
S3150000FCD08000F8F7CFFE641C102CE8D34FF001101B
S3150000FCE049490860002049490860494908600120DF
S3150000FCF0F8F73FFEE87910F0400F06D04548008837
S3150000FD0040F001004349088009E04248008820F09D
S3150000FD1001004049088002E06888054427E022E0A7
S3150000FD20EE7820E058E027E0E6B9A87800F08F04E6
S3150000FD3014F0800F05D004F00F014FF48030884096
S3150000FD4001E00120A04007462F48006838432E49AD
S3150000FD5008602846F8F768FE2046F8F774FE204645
S3150000FD60F8F708FE00BF00BF2878054400BF2878D2
S3150000FD7000287FF47CAF26E000201F49087001248C
S3150000FD8014E00120A04020490968084202D020461C
S3150000FD90F8F770FE4FF48030A0401B49096808420E
S3150000FDA003D044F08000F8F765FE641C102CE8D3FD
S3150000FDB04FF00110144908600020144908601449E6
S3150000FDC00860F8F7D6FD074880780B49097888421D
S3150000FDD001D0002042E701E000203FE700BF0120FC
S3150000FDE03CE7000004E1FF1FA5090100F9E0FF1F41
S3150000FDF0CE0A0100490B0100EBE0FF1FF8E0FF1FF0
S3150000FE0008E0FF1FA6090100ECE0FF1FF0E0FF1F5E
S3150000FE10F4E0FF1FE8E0FF1F2DE9F05F0027B8467A
S3150000FE20BB46B9464948007800F01F0001287CD13E
S3150000FE304748007810B90020BDE8F09F4FF0000A4F
S3150000FE404448007828B944480078012801D10020A8
S3150000FE50F2E74148007808B9404C00E0404C6CE0BD
S3150000FE606078022804D004280BD0052861D11EE052
S3150000FE70607937490978884202D0608804445CE09A
S3150000FE8057E0A77894F803804FF000092F480079CF
S3150000FE90B8420BD12D488078404507D14FF0010A72
S3150000FEA0304810F807B0014601F8078041E02748BE
S3150000FEB00079B8423CD1A07800F08F0616F0800F8A
S3150000FEC005D006F00F014FF48030884001E0012094
S3150000FED0B04005461D488078404515D12248006847
S3150000FEE028432149086021480068A8431F49086043
S3150000FEF02046F8F799FD3046F8F7A5FD3046F8F7A5
S3150000FF0039FD49EA050913E0D84511D119EA050F6B
S3150000FF100ED115480068A8431349086013480068C5
S3150000FF20A84312490860304600E00AE0F8F7A2FD4F
S3150000FF3000BF00BF2078044400BF207800288FD17E
S3150000FF4001E0002078E700BF504675E704E1FF1F97
S3150000FF50EBE0FF1FA5090100F9E0FF1FCE0A010033
S3150000FF60490B010008E0FF1FECE0FF1FF0E0FF1F58
S3150000FF7002E008C8121F08C1002AFAD1704770476C
S3150000FF80002001E001C1121F002AFBD1704710B505
S3150000FF90002A06DA22F00042D21D22F007031022C0
S3150000FFA003E0D21C22F003030C2213B19C188C42EE
S3150000FFB001D9012010BD024401448360C0E900213B
S3150000FFC0C91AD018884202D810600246F9E7002004
S3150000FFD0106010BD08480068C0010BD507480068CE
S3150000FFE0C00707D0054880380068002802DA0449AF
S3150000FFF00120087070470000FCED00E0800E00E074
S3150001000020E1FF1F4FF06042D36F002BFCD0C36A83
S31500010010D367D36F002BFCD0C07840EA0120A2F849
S315000100207C0070474FF06041CA6F002AFCD081F80E
S315000100307C0070470A460146074810B500EB82006E
S3150001004050F8040C002805D000F05EFABDE8104017
S3150001005000F04ABA10BD00005CF3FF1F07480168B3
S315000100604FF0E020416100218161072101610448CF
S31500010070016841F07F41016040177047880901001E
S3150001008020ED00E0704750E8001F31B10B6840E8F1
S315000100900032002AF7D108467047BFF32F8FFAE7DF
S315000100A070B50D46002812D04FF6FF71084C8842F4
S315000100B004D222680146104600F052FA20684570C3
S315000100C0044800F0F5F8BDE8704000F001BB70BDD2
S315000100D014E1FF1F1414002070B51A4DE8680028BA
S315000100E02ED0A88A401EA882002623E0A06838B137
S315000100F061684160606810B1A16881606660A66050
S3150001010010482146183800F04FFAA08AA882607874
S31500010110042804D10C49E08A09880844A0820120F8
S31500010120607084F82000E068E860E06808B1056165
S31500010130E6602661A88A002802D1EC68002CD5D198
S3150001014070BD00002C1400201CE1FF1F70B50400D7
S315000101500FD00D4DA17801262868827891420CD9DD
S3150001016000F03EFA286846702046BDE8704000F06F
S31500010170AFBA064800F09CF8F7E766702146BDE87D
S315000101807040024800F010BA14E1FF1F1414002059
S315000101900321FFF785BF000001480068408B7047C7
S315000101A014E1FF1F10B50446008B084320836278D3
S315000101B0618B062A16D0052A17D1084215D001EA05
S315000101C00002628388432083204600F013FA01204F
S315000101D06070022084F820002146BDE810400348E3
S315000101E000F0E2B931EA0002ECD010BD141400208F
S315000101F0024670B5154800EB810050F8044C002CFE
S3150001020022D0208B104320836178658B062918D074
S31500010210052919D1284217D005EA00016183A843AF
S315000102202083204600F0E6F9208BA8432083012095
S315000102306070022084F820002046BDE87040FFF778
S3150001024085BF35EA0001EAD070BD00005CF3FF1FEF
S3150001025070B503460D480D460468208B42B133EA5A
S31500010260000101D0062009E098432083022070BDD9
S3150001027010EA030201D06283F6E70520C1B2638367
S315000102802846FFF70DFF012070BD000014E1FF1F96
S31500010290814202D342688A4201D80120704750E860
S315000102A0002F0A6040E80012002AF8D100207047AA
S315000102B00146406842684A600B780022022B05D04D
S315000102C0012B03D0032B01D04260704743680BB169
S315000102D0996042608260704770B5044600201546F9
S315000102E0207001226270A1706060A060E0602061F0
S315000102F0A082E0822083608384F8200084F82100B4
S31500010300608C18B90448FFF7BEFEA0622946204654
S31500010310BDE8704000F002B8B0E3FF1F10B5428C93
S31500010320920803D10F4A1288C2F38D02836A03EB46
S315000103308202530700D5121F403A4FF08073C2E97B
S315000103400E1300234FEA030442F823405B1C0E2BD5
S31500010350FAD3C36913624262C162806A02490160CB
S3150001036010BD000080090100A52E5AE20349044A86
S315000103700968C882128810448882704714E1FF1FF9
S315000103801CE1FF1F0848016808488A8A0088CB8A51
S31500010390A2EB00001A4480B28A82010402D404212D
S315000103A0FFF77EBE7047000014E1FF1F1CE1FF1F2F
S315000103B02DE9F0410F4604464168002004F10C0680
S315000103C021B1617802291AD0A189A9B3A189E2894B
S315000103D0914246D2218904EB81010F61D6E85F1F64
S315000103E0491CC6E8521F002AF8D12189491C89B245
S315000103F02181E289914200D12081BDE8F081074641
S3150001040060702046FFF754FF80F820702189054669
S3150001041004EB8101C0690861D6E85F0F401CC6E89C
S31500010420510F0029F8D12089401C80B22081E18931
S3150001043088420BD1278109E0FFE72046FFF738FF05
S315000104400546C0690421076085F8201001206870FF
S31500010450284600F0CFF82946BDE8F041034800F0F0
S31500010460A3B8BDE8F0410320F8F797B914140020AA
S3150001047070B51A4801210068417000F0B1F8184DB5
S315000104806C7816E005EBC40148680278E2B1012AEE
S315000104901FD000F0C9F8E878641C844200D100241A
S315000104A00F48801CD0E84F1F491EC0E8421F002A92
S315000104B0F8D1A8780028E5D16C700A48FFF7F8FE54
S315000104C0BDE8704000F004B9098989B2FFF76AFEF8
S315000104D0E1E78968FFF76CFFDDE7000014E1FF1F24
S315000104E038F3FF1F141400200548017811B10121CA
S315000104F04170704703494FF0805008607047000013
S31500010500D400002004ED00E0F0B4144A941CD57820
S315000105104FEA0206D4E84F3FAB4202D1BFF32F8F19
S315000105200EE05B1CC4E8473F002FF3D1D6E84F3FEE
S315000105305C1CAC4200D10024C6E8474F002FF5D120
S31500010540D4789C4205D902EBC302C2E90101F0BC91
S315000105507047F0BC0220F8F720B9000038F3FF1FFE
S31500010560104A10B5D368ABB113469B8A03E08CB130
S315000105702246A48A2344D4688B42F8D3C460D0604F
S315000105800261C46804B12061591A8182908A401AB5
S31500010590908210BD0024C460D060C91A02619182A4
S315000105A0848210BD2C14002030B502780023022A63
S315000105B003D0012A01D0032A00D101238C7800E05F
S315000105C01046426812B19578A542F9D24A60416057
S315000105D01BB102B19160886030BD0020FBE70000CD
S315000105E003494A6842600022826048607047000001
S315000105F01414002010B5016900290ED0C268CA6022
S31500010600C36800223BB18B8A848A23448B82C368E8
S315000106101961C26000E08A82026110BD0222027085
S31500010620002242604180704710B5416879B1FFF7F9
S315000106303FFE0446FFF7DEFF01206070032084F8C9
S3150001064020002146BDE810400348FFF7ADBF4188B1
S31500010650491C418010BD00001414002010B54168EA
S3150001066089B1FFF725FE0446032084F820002046C1
S31500010670FFF7C0FF2046FFF769FD0549002009681D
S3150001068081F8200002E04188491C4180002010BD0C
S3150001069014E1FF1F10B542880C461AB1521E428062
S315000106A0002010BD34B1094A4368116823B1FFF730
S315000106B07BFF06E0012010BD416011680023C1E9FE
S315000106C0013007212046FFF7EBFCF3E714E1FF1F9A
S315000106D00749022248604270064A1278002A05D06C
S315000106E006C98A4202D0C078FFF79CBC7047000059
S315000106F014E1FF1F20E1FF1F2DE9F047164688464A
S315000107008146FFF767FC002004463E4A3E4902E067
S3150001071042F82040401C0B889842F9D33B483022CE
S3150001072001883B48FFF733FC3A48008880B240F025
S315000107300042394801683948FFF729FC3848082240
S31500010740018838480068FFF722FC374FFF25374AF2
S31500010750FD707C8400213846FFF7BEFD3448042134
S315000107600170446033480170C46004618482786A10
S315000107702030F7F74FFE3048314907600220787084
S315000107802E48047044700978C170F8F708F82D48AE
S31500010790016841F47F0101600068290601EA002031
S315000107A02849C0431439B0FA80F00968C0F108003D
S315000107B0C1F30221814200DB481C2249091F0B6853
S315000107C06FF08072824063F317020A60FFF746FCFE
S315000107D01D49002808600CDB1C49455400F01F0226
S315000107E00121914040114FF0E02202EB8000C0F858
S315000107F00011324641464846BDE8F047002300F065
S315000108006BB800005CF3FF1F7C0901009809010029
S3150001081030E1FF1F800901009C090100B0E3FF1FC1
S31500010820A209010000E0FF1FECF4FF1F95870000FD
S31500010830141400202C14002014E1FF1F38F3FF1FAD
S31500010840A009010020ED00E0D800002000E400E04E
S315000108500B4810B5006801214170FFF7C1FEF7F79B
S315000108609FFF08480168491C0160FFF735FC00F04D
S3150001087013F80548FFF71CFDBDE81040FFF728BF38
S3150001088014E1FF1F1CE1FF1F14140020014800683A
S31500010890704700001CE1FF1F70B50D4C2068002851
S315000108A015D0A0880B4E401EA0800AE0E888F7F715
S315000108B073FFA888A0802868206029463068FFF762
S315000108C0E7FCA088002802D12568002DEED170BD75
S315000108D024E1FF1F00E0FF1F2DE9F0411E461746E8
S315000108E080460C4611F0FF0F00D14C1C1A48FFF749
S315000108F0CAFB05002DD0C4F30F20AF626884E1B2B4
S3150001090042462846EE61FFF7E7FC012413481449E5
S3150001091006E000BF00EB840252F8042C22B1641CED
S315000109200A889442F6D9002400EB8400E6B240F826
S31500010930045C0C48EE70007818B101212846FFF7D7
S3150001094061FB2846FFF702FC0748006880F8206033
S315000109502046BDE8F081000030E1FF1F5CF3FF1F78
S315000109607C09010020E1FF1F14E1FF1F0248006816
S31500010970002800D0C078704714E1FF1F0D00000069
S31500010980B80105000A000000FF520700010000003F
S3150001099010270000000000007C020000880F000004
S315000109A00400000000000400040803010100010026
S315000109B04000400004000101400040000100000227
S315000109C0020040000002010203040440800000000E
S315000109D00000000000000000000000000000000010
S315000109E0000000000000000000000000C9D800005F
S315000109F000000000000000000000000000000000F0
S31500010A0000000000000000000000000000000000DF
S31500010A1000000000000000000000000000000000CF
S31500010A2000000000000000000000000000000000BF
S31500010A3000000000000000000100000035930000E6
S31500010A405993000081DC0000BBE50000C7F30000FC
S31500010A5061D70000C7D700000000000000000000B9
S31500010A60000000000000000000000000000000007F
S31500010A70000000000000000000000000000000006F
S31500010A80000000000600FF0901A101150026FF0074
S31500010A907508954009018102954009019102950168
S31500010AA00901B102C0002100120110010200000873
S31500010AB0280D04020001010203010A0610010000CB
S31500010AC0000801000A0600020000000801000902F0
S31500010AD07A0004010080FA090400000208065007A2
S31500010AE007058202400000070502024000000904D2
S31500010AF00100010202010005240010010524010381
S31500010B0002042402060524060102070583031000D8
S31500010B100209040200020A0000000705040240005F
S31500010B2000070584024000000904030002030000D7
S31500010B300609210001000122210007058103400069
S31500010B400107050103400001000000000403090438
S31500010B500A034D004200450044001E034D004200B9
S31500010B6045004400200043004D0053004900530056
S31500010B702D004400410050001603410030003000B2
S31500010B8030003000300030003000300031002203E8
S31500010B906D0062006500640020005300650072006C
S31500010BA0690061006C00200050006F007200740043
S31500010BB0040320001E034D004200450044002000AE
S31500010BC043004D005300490053002D0044004100ED
S31500010BD0500010035500530042005F004D005300C2
S31500010BE04300EB3C904D53444F53352E30000201E8
S31500010BF001000220000002F00100010001000000D6
S31500010C00000000000000000029741902274D6265EA
S31500010C106420555342202020464154313220202061
S31500010C2033C98ED1BCF07B8ED9B800208EC0FCBDF5
S31500010C30007C384E247D248BC199E83C01721C83CB
S31500010C40EB3A66A11C7C26663B07268A57FC75068D
S31500010C5080CA0288560280C31073EB33C98A4610D4
S31500010C6098F7661603461C13561E03460E13D18BC0
S31500010C707611608946FC8956FEB82000F7E68B5E40
S31500010C800B03C348F7F30146FC114EFE61BF00009A
S31500010C90E8E600723926382D741760B10BBEA17DC6
S31500010CA0F3A66174324E740983C7203BFB72E6EBEF
S31500010CB0DCA0FB7DB47D8BF0AC9840740C487413BA
S31500010CC0B40EBB0700CD10EBEFA0FD7DEBE6A0FC5B
S31500010CD07DEBE1CD16CD19268B551A52B001BB001D
S31500010CE000E83B0072E85B8A5624BE0B7C8BFCC78E
S31500010CF046F03D7DC746F4297D8CD9894EF2894E51
S31500010D00F6C606967DCBEA030000200FB6C8668BB1
S31500010D1046F86603461C668BD066C1EA10EB5E0F89
S31500010D20B6C84A4A8A460D32E4F7E20346FC135630
S31500010D30FEEB4A525006536A016A10918B46189689
S31500010D409233D2F7F691F7F64287CAF7761A8AF204
S31500010D508AE8C0CC020ACCB80102807E020E750474
S31500010D60B4428BF48A5624CD136161720B4075012E
S31500010D7042035E0B497506F8C341BB000060666A13
S31500010D8000EBB04E544C44522020202020200D0A66
S31500010D9052656D6F7665206469736B73206F72207F
S31500010DA06F74686572206D656469612EFF0D0A4472
S31500010DB069736B206572726F72FF0D0A50726573EB
S31500010DC07320616E79206B657920746F207265736B
S31500010DD0746172740D0A00000000000000ACCBD8EB
S31500010DE055AAF0FFFFFFFFFF000000000000000012
S31500010DF00000004641494C20202020545854201818
S31500010E00B174768E418E4100008E768E41040007C4
S31500010E100000004D424544202020202020202800AB
S31500010E2000000000000000000085758E41000000F2
S31500010E30000000412E0066007300650076000F0079
S31500010E40DA65006E0074007300640000000000FFA4
S31500010E50FFFFFF46534556454E7E312020201200A6
S31500010E60477D758E418E4100007D758E41020000E1
S31500010E7000000042650072005F0069006E000F000D
S31500010E80A86400650078000000FFFFFFFF0000FF77
S31500010E90FFFFFF012E006D006500740061000F0069
S31500010EA0A864006100740061005F006E00000065C7
S31500010EB00076004D45544144417E312020202200D8
S31500010EC03285758E418E41000085758E4100000088
S31500010ED0000000412E0054007200610073000F00F3
S31500010EE0256800650073000000FFFFFFFF0000FF9B
S31500010EF0FFFFFF5452415348457E312020202200F6
S31500010F003285758E418E41000085758E4100000047
S31500010F100000004D4245442020202048544D201811
S31500010F20B174768E418E4100008E768E41030001AA
S31500010F30010000002E202020202020202020203209
S31500010F4000477D758E418E41000088758E410200F5
S31500010F50000000002E2E20202020202020202010FE
S31500010F6000477D758E418E4100007D758E410000E2
S31500010F70000000004E4F5F4C4F47202020202020CC
S31500010F80083285758E418E41000085758E410000BF
S31500010F90000000003C212D2D206D626564204D6905
S31500010FA063726F636F6E74726F6C6C6572205765D6
S31500010FB0627369746520616E642041757468656E3B
S31500010FC07469636174696F6E2053686F72746375B7
S31500010FD074202D2D3E0D0A3C68746D6C3E0D0A3C45
S31500010FE0686561643E0D0A3C6D65746120687474C0
S31500010FF0702D65717569763D2272656672657368D5
S315000110002220636F6E74656E743D22303B207572CB
S315000110106C3D687474703A2F2F6D6265642E6F7221
S31500011020672F6465766963652F3F636F64653D402D
S3150001103041222F3E0D0A3C7469746C653E6D6265F2
S315000110406420576562736974652053686F727463AF
S3150001105075743C2F7469746C653E0D0A3C2F686586
S3150001106061643E0D0A3C626F64793E3C2F626F6497
S31500011070793E0D0A3C2F68746D6C3E0D0A0D0A000F
S3150001108030313233343536373839414243444546B7
S315000110900000000000BE0AE00D782D066840082415
S315000110A0400000D35840641EFAD1491C521E002A42
S315000110B0F2D170472F4910B5494408602E480021E6
S315000110C001602F482D4A4844026001224160920482
S315000110D082609202C26005229206426101221203D7
S315000110E08261024620321170491E416200F029F9DF
S315000110F0002800D0012010BD00207047214A08B504
S315000111007A44490300920A0C01461D4800234844CB
S3150001111000F0B7F9002800D0012008BD10B5194923
S31500011120794417482039484400F091F8002800D046
S31500011130012010BD10B5134B7B4401461048012216
S31500011140383B9202484400F0B4F8002800D0012050
S3150001115010BD38B50C460B49794458390091014602
S31500011160074813462246484400F048F9002800D0B3
S31500011170012038BD04000000008104400000024047
S31500011180080000008500000070B5044600680025CF
S3150001119003781B06FCD57023037000203AE0030098
S315000111A000F060FA0C070B0F13171B1F23272B2FB9
S315000111B0333626681378F3712AE026685378B371BB
S315000111C026E026689378737122E02668D378337116
S315000111D01EE026681379F3721AE026685379B37212
S315000111E016E026689379737212E02668D379337212
S315000111F00EE02668137AF3730AE02668537AB3730E
S3150001120006E02668937A737302E02668D37A33730D
S31500011210401CC0B28842C2D921688020087003E010
S31500011220606A411C00D08047206800780006F7D527
S3150001123020680078810601D5042506E0C10601D59E
S31500011240082502E0C00700D01025284670BD08B564
S315000112500B46442269460A706A460021984708BD32
S3150001126038B514468A0702D0FF20013038BD4368DD
S315000112708B4203D882689A188A420DD8C2688A427C
S3150001128003D80369D3188B4201D8022038BD891AC5
S315000112900122D205891800E0C91A08226B461A7084
S315000112A00A0C5A700A0A9A70D9706A460321A04735
S315000112B038BDFFB581B01546019A0127526800264F
S315000112C04819BF028A4204D8019B9B68D3188342FE
S315000112D00FD2019AD2688A4204D8019B1B69D3189E
S315000112E0834201D2022629E0881A0121C905441840
S315000112F000E08C1A3946204600F007F9002902D091
S31500011300FF2601361AE03946284600F0FEF8002984
S3150001131012D0012612E0092069460870200C487097
S31500011320200A8870CC70049B6A460321019898476D
S31500011330060003D1ED1BE419002DECD1304605B0B2
S31500011340F0BDF0B5016800240A781206FCD57022BA
S315000113500A7002680321D171016880228A710368CB
S31500011360002159710568FC232B710368D973036841
S315000113701A70026813781B06FCD5557A127A17077C
S3150001138001223F0FD20356103B0000F06BF9100902
S315000113900B0E1009090909101F0E0909090909117E
S315000113A0026105E003225203FAE7066100E00161EA
S315000113B02A07120F130000F055F9100C0C0C0F122E
S315000113C015181B1D1F0C0C0C0C0C0C0D01225203C5
S315000113D0E6E7C1612046F0BD0121C902F9E7012115
S315000113E08902F6E701214902F3E7FF210131F0E71E
S315000113F08021EEE74021ECE72021EAE7FEB507462A
S3150001140016461D4600208A198B0702D0FF2001309F
S31500011410FEBDB30701D00120FEBD7B688B4203D818
S31500011420BC681C1994420DD2FB688B4203D83C69F7
S315000114301C19944201D20220FEBD0122C91AD2050D
S315000114408C181BE0CC1A19E0062069460870200C9E
S315000114504870200A8870CC70E8780871A8784871BD
S31500011460687888712878C871089B6A4607213846CA
S3150001147098470028E0D1241D361F2D1D002EE3D1EB
S31500011480FEBDFEB5154604464268A80040181E4634
S315000114908A4203D8A368D3188B4208D8E3688B42E3
S315000114A003D82769DB198B4201D80220FEBD82428F
S315000114B005D8A368D318834201D38F1A0AE0E268DC
S315000114C0824203D92369D3188342EED3881A0121B4
S315000114D0C90547180421384600F017F8002902D03B
S315000114E0FF200130FEBD012069460870380C4870A6
S315000114F0380A8870CF70280A08714D718E71089B61
S315000115006A46062120469847FEBD002203098B4202
S315000115102CD3030A8B4211D300239C464EE003468B
S315000115200B433CD4002243088B4231D303098B423F
S315000115301CD3030A8B4201D394463FE0C3098B4275
S3150001154001D3CB01C01A524183098B4201D38B01CE
S31500011550C01A524143098B4201D34B01C01A524171
S3150001156003098B4201D30B01C01A5241C3088B42B6
S3150001157001D3CB00C01A524183088B4201D38B00A1
S31500011580C01A524143088B4201D34B00C01A524143
S31500011590411A00D201465241104670475DE0CA0F1A
S315000115A000D04942031000D34042534000229C46DA
S315000115B003098B422DD3030A8B4212D3FC228901E4
S315000115C012BA030A8B420CD3890192118B4208D3BA
S315000115D0890192118B4204D389013AD0921100E01C
S315000115E08909C3098B4201D3CB01C01A5241830930
S315000115F08B4201D38B01C01A524143098B4201D35D
S315000116004B01C01A524103098B4201D30B01C01A87
S315000116105241C3088B4201D3CB00C01A5241830801
S315000116208B4201D38B00C01A5241D9D243088B4257
S3150001163001D34B00C01A5241411A00D201466346FA
S3150001164052415B10104601D34042002B00D549425E
S31500011650704763465B1000D3404201B50020C04687
S31500011660C04602BD30B47446641E2578641CAB4284
S3150001167000D21D46635D5B00E31830BC18470000CD
S31500011680FEFFFFFF20000020640000200300002071
S315000116906800002088000020A0000020BE00002075
S315000116A0FFFFFFFF4000000001000020EC050020C5
S315000116B0001000200020002000000020EC050000A2
S315000116C0941001000002000085170100E9B6000030
S315000116D08BB30000FDB30000F3B0000071B1000050
S315000116E041B400008416010000040000303230309D
S315000116F03738613063643732312E30004D4245440C
S31500011700202020206D6963726F636F6E74726F6C37
S315000117106C65757220312E302000424144204558B7
S3150001172054454E53494F4E2046494C450053574464
S3150001173020504F525420494E20555345005357448B
S31500011740204552524F520042414420535441525473
S3150001175020534543544F52004E4F5420434F4E534E
S315000117604543555449564520534543544F5253001A
S315000117705245534552564544204249545300544913
S315000117804D454F555400303230300000CC17010022
S3150001179000E0FF1F2C0100003CF8000020180100AA
S315000117A000000020DC00000070FF0000201801008E
S315000117B02CE1FF1FF013000080FF0000FC18010060
S315000117C0DC0000206C15000080FF0000410415FCC0
S315000117D016011BE20B181A0208130D01320B1AF23D
S315000117E0084114130E011A200B4B330F101A34083B
S315000117F0326013280E2A203032071A011B143D17B6
S31500011800011A1A041A58041A2D041A70041A4704E4
S315000118101A7E040140E9424380250A11081A014A49
S31500011820006CDC0255555555000000000000000013
S3150001183000000000010000000000000000000000A0
S315000118400000000000000000000000000000000091
S3150001185000000000000000008617010000000000E3
S31500011860000000000000000000000000C816010092
S315000118700000000000000000000000000000000061
S315000118800000000000000000000000000000000051
S315000118900000000000000000000000000000000041
S315000118A00000000000000000000000000000000031
S315000118B00000000000000000000000000000000021
S315000118C00000000000000000000000000000000011
S315000118D00000000000000000000000000000000001
S315000118E000000000000000000000000000000000F1
S311000118F0000000000000000000000000E5
S7050000840175
